:020000040800F2
:10000000D810002005010008FF3700080D2900085E
:10001000FD3700083D0F00081D61000800000000CA
:100020000000000000000000000000005147000830
:10003000CB1A0008000000006D3D0008394A000896
:100040001F0100086D3B00081F0100081F01000888
:100050001F0100081F0100081F0100081F01000800
:100060001F0100081F0100081F0100081F010008F0
:100070001F0100081F0100088D1500081F0100085E
:100080001F0100081F010008410700081F010008A8
:100090001F0100081F0100081F0100081F010008C0
:1000A000A94A0008894B00081F0100081F01000829
:1000B0008D4B00087D4E0008D95000081F01000834
:1000C0001F0100081F0100081F0100081F01000890
:1000D0001F010008155C00081F0100081F0100082F
:1000E0001F0100081F0100081F010008DFF810D0E1
:1000F00000F0E8FA0048004745720008AFF30080BE
:10010000D81000200648804706480047FEE7FEE773
:10011000FEE7FEE7FEE7FEE7FEE7FEE7FEE7FEE7B7
:10012000594A0008ED0000082DE9F0410024061BA3
:10013000254671F1000605DA01240027D0EB0700FF
:1001400067EB0101161E73F1000605DA0027D2EBFA
:100150000702012567EB030300F0D0F986460E463F
:1001600017469C46AC4204D00025D0EB050E65EB4B
:10017000010624B10020D2EB000760EB030C7046AF
:1001800031463A466346BDE8F08140EA01039B07E9
:1001900003D009E008C9121F08C0042AFAD203E0FC
:1001A00011F8013B00F8013B521EF9D2704780EA7A
:1001B000010210B502F00043400022D04A001FD0D7
:1001C000010E01EB1261C0F35600C2F3560240F477
:1001D000000042F40002A0FB022000047F39140456
:1001E00000D0401C50EA124001D44000491EC2B267
:1001F0000C0604EBD010401C4008802A02D003E01B
:10020000002010BD20F00100002900DA0020184372
:1002100010BD2DE9FE4F81EA030404F0004421F0F3
:10022000004100944FF0000B23F0004350EA01041A
:100230005ED052EA03045BD0C3F30A54C1F30A55FB
:100240002C44A4F2F3340194A0FB0254C1F3130133
:1002500041F48011C3F3130343F4801301FB024400
:1002600000FB034E840A970A44EA815447EA835705
:10027000A4FB076802958D0A05FB07854FEA932CBE
:1002800004FB0C542705029D4FEA065847EA16372F
:10029000B5EB08056EEB070C870E920E47EA811747
:1002A00042EA8312A7FB0201B6EB0B0164EB0004E8
:1002B0002B0D43EA0C335E1844EB1C50DA465146D2
:1002C000E7FB0201C5F313044FEA0B3343EA14536F
:1002D0004FEA0432019C43EA0603A4F10C040294A1
:1002E000009CCDE900B400F09FF903B0BDE8F08FA9
:1002F00000200146F9E72DE9F04D81EA030404F0FE
:10030000004B21F0004514464FF0000A23F0004155
:1003100050EA050220D054EA01021DD0C5F30A5765
:100320000246C5F31303C1F31300C1F30A5640F4A8
:10033000801543F48013A7EB0608101BD64608F27D
:10034000FD3873EB050002D308F1010801E09218B3
:100350005B41B8F1000F03DA00200146BDE8F08DE3
:1003600000204FF48011064684460EE0171B73EB05
:10037000050705D3121B63EB050306434CEA010C8A
:1003800049084FEA300092185B4150EA0107EDD16D
:1003900052EA030012D082EA040083EA050108430E
:1003A00005D0101BAB4106D20122002306E000223B
:1003B0004FF0004302E06FF0010253101AEB060009
:1003C0004CEB085110EB0A0041EB0B01BDE8F04D7E
:1003D00000F01BB970B521F0004303430CD0C1F30A
:1003E0000A550024D5EB040564EB0403D617AD1AB7
:1003F000B34102DB0020014670BD201841EB0251E1
:1004000070BDC10F80EAE0700844CA07962300213E
:1004100000F0CDB896230022114600F0C8B80EB502
:10042000C10F80EAE0700844CA07002140F233435C
:100430008DE80E000A460B4600F0F6F803B000BD4A
:100440000EB540F2334102910021CDE900110A4678
:100450000B4600F0E9F803B000BD00F0004220F0C8
:100460000040C10DC0F3160040F400007F2901DAFE
:1004700000207047962903DCC1F19601C84001E0D5
:1004800096398840002AF4D04042704770B5C1F3D5
:100490000A5201F000450024C1F3130140F2FF337A
:1004A00041F480119A4201DA002070BD40F23343DA
:1004B0009A42A2F2334203DC524200F05FF800E0BD
:1004C00090402C43F1D0404270BDC1F30A5210B5A8
:1004D000C1F3130140F2FF3341F480119A4201DA73
:1004E000002010BD40F233439A42A2F2334203DCB3
:1004F000524200F043F810BD904010BD2DE9F05F6E
:100500000546002092469B46884606468146402482
:100510001BE0284641464746224600F02FF8534646
:100520005A46C01A914110D311461846224600F08F
:1005300016F82D1A67EB01084F46224601200021CC
:1005400000F00DF817EB00094E41201EA4F1010444
:10055000DFDC484631462A464346BDE8F09F202A64
:1005600004DB203A00FA02F1002070479140C2F10A
:10057000200320FA03F3194390407047202A04DB3C
:10058000203A21FA02F00021704721FA02F3D0400C
:10059000C2F1200291400843194670470029A8BFC4
:1005A0007047401C490008BF20F00100704710B49C
:1005B000B0FA80FC00FA0CF050EA010404BF10BC51
:1005C000704749B1CCF1200421FA04F411FA0CF17E
:1005D00018BF012121430843A3EB0C01CB1D4FEAB7
:1005E00000614FEA102042BF002010BC704700EBB2
:1005F000C35010440029A4BF10BC7047401C4900E0
:1006000008BF20F0010010BC704710B5141E73F134
:10061000000408DA401C41F1000192185B411A43C2
:1006200001D120F0010010BD2DE9F04D92469B460E
:1006300011B1B1FA81F202E0B0FA80F220329046B4
:10064000FFF78DFF04460F4640EA0A0041EA0B011E
:1006500053465A46084313D0114653EA010019D0B5
:10066000C8F140025046FFF789FF05460E46504646
:1006700059464246FFF773FF084305D0012004E0C6
:1006800020463946BDE8F08D0020054346EAE07675
:100690002C4337430A986305E40AA0EB08000022C4
:1006A000FD0A44EA47540A3002D500200146E9E732
:1006B000010510196941DDE9084500196941BDE8E6
:1006C000F04DA2E7064C074D06E0E06840F001035C
:1006D00094E8070098471034AC42F6D3FFF70AFDC0
:1006E000689200088892000870B58C1810F8015BB9
:1006F00015F0070301D110F8013B2A1106D110F8BB
:10070000012B03E010F8016B01F8016B5B1EF9D1BE
:100710002B0705D40023521E0DD401F8013BFAE744
:1007200010F8013BCB1A921C03E013F8015B01F8AF
:10073000015B521EF9D5A142D8D3002070BD000044
:1007400070B54F4C4FF490652946204600F01BFAD7
:10075000002866D02946204600F0A8F849490888B4
:10076000401C08800121204600F0ECFA464942F284
:100770001072B1F85000904202D2401CA1F8500013
:1007800006F03CFF05F03EF8404DB5F91410B5F900
:10079000120005F011FE3E4CA5F84E002080A16825
:1007A00020468847A088A5F8500003F091F807F08C
:1007B00027F8384E384C3078082833D045F6AC301E
:1007C000606042F6EF60A06042F2C400E06033482F
:1007D000008A2080208E6080A16B2F488847208E61
:1007E00069882F4C08444FF6FF7101EA8000688643
:1007F000207A4FF0000540071DD501F0F5FA294990
:1008000049F6A2400880284840F21A62C188491C73
:1008100089B2C180914204D3A16821F00401A16092
:10082000C58070BD41F2130060604FF48060A0602D
:1008300040F61B50CAE730780A281BD2DFE800F0E8
:100840001A0616050A050D1A1114EAE7BDE87040EC
:1008500005F056BF07F0EEFE08E0BDE8704002F07C
:1008600081BD06F0C7FA01E007F022F9BDE870404B
:1008700007F01EB900F0FAFB84F8B65070BD000016
:1008800000240140FC060020400100206000002000
:1008900018070020F3060020D0000020F0010020FF
:1008A0009C020020442C01401C0900206FEA112109
:1008B000016070470029816802D041F0010101E028
:1008C00021F00101816070470029816802D041F464
:1008D000807101E021F48071816070472DE9F04161
:1008E000824E92B0304600F00BF90BA800F039FAB6
:1008F00001214FF4C06003F0EFFA00248DF831407D
:100900004FF46020CDE90D044FF4A0204FF009080A
:100910000B9001278DF83C808DF830700BA9304684
:1009200000F080F9724D8DF831408DF830708DF8FF
:100930003C700BA9284600F075F901231A460F21D7
:10094000304600F0C0F9022201231146304600F083
:10095000BAF9012303220021304600F0B4F9012343
:1009600004221946304600F0AEF9012305220B217E
:10097000304600F0A8F9012306220421304600F099
:10098000A2F9012307220821304600F09CF9012337
:1009900008220321304600F096F9012309220A219A
:1009A000304600F090F90121304600F084F9012131
:1009B000284600F080F901231A460521304600F050
:1009C00055F901231A460621284600F04FF9002167
:1009D000304600F0CBF84FF4E041284600F0C6F86E
:1009E0000121304600F0B8F80121284600F0B4F8A3
:1009F0000121304600F0A6F80121284600F0A2F8B7
:100A00000121304600F09EF90121284600F09AF9B4
:100A100040F61451374804F036FE12208DF840009D
:100A200002208DF841008DF842408DF8437010A8E7
:100A300002F012FF01224FF49061304600F0E8F816
:100A400001213046FFF740FF01213046FFF732FF1A
:100A500001212846FFF72EFF304600F06EF93046A0
:100A600000F09FF80028FAD1304600F075F93046C2
:100A700000F082F80028FAD1284600F05EF92846F6
:100A800000F08FF80028FAD1284600F065F92846D2
:100A900000F072F80028FAD10121084603F0F8F9B5
:100AA000154D284600F0AEFD684600F056FE0F4892
:100AB00001A94C300090114881E811018020CDE956
:100AC00004404000069080000790202008904FF4DA
:100AD0004050CDE909046946284600F021FE012175
:100AE000284600F083FD12B0BDE8F08100240140EB
:100AF00000280140002C014008000240AC02002008
:100B00000D4910B5884202D1012144150AE00B4974
:100B1000884202D10121041504E0094988420AD122
:100B20000121CC03204603F0E3F92046BDE8104044
:100B3000002103F0DDB910BD002401400028014070
:100B4000003C01400029816802D041F4801101E09D
:100B500021F48011816070470029816802D041F43E
:100B6000004101E021F4004181607047826822F475
:100B7000E0420A43826070470146002089684907C5
:100B800000D50120704710B50246002054680B0ABA
:100B9000C9B20C401168194202D0002C00D00120CB
:100BA00010BD014600208968090700D50120704763
:100BB00038B501211C2003F08FF9FF20ADF80000AB
:100BC00000248DF8034003258DF8025069460D4836
:100BD00001F00CFB0120ADF800008DF803408DF80A
:100BE00002506946084801F001FB2320ADF80000DF
:100BF0008DF803408DF802506946044801F0F6FA7A
:100C000038BD000000080140000C01400010014008
:100C1000002A4268C9B201D00A4300E08A43426018
:100C20007047000010B542680E4B0C791A400B68F3
:100C300042EA04221343436083680B4A1340D1E91C
:100C4000024222434C7943EA44031A438260C26A57
:100C5000097C22F47002491EC9B242EA0151C16204
:100C600010BD0000FFFEF0FFFDF7F1FF70B5072497
:100C700009290AD9C568A1F10A0606EB4606B4405F
:100C8000A543B3401D43C56007E0056901EB41067C
:100C9000B440A543B3401D430561836BC3F30154C6
:100CA000121B921C02EB82041F22A2409343A1401C
:100CB0000B43836370BD826B491E22F4401242EAEB
:100CC00001518163704770B5072409290AD9C568A5
:100CD000A1F10A0606EB4606B440A543B3401D4306
:100CE000C56007E0056901EB4106B440A543B34088
:100CF0001D4305611F23072A09D2446B521E02EBD4
:100D0000820293409C4391400C43446370BD0D2A82
:100D100009D2046BD21F02EB820293409C439140A4
:100D20000C43046370BDC46A0D3A02EB8202934027
:100D30009C4391400C43C46270BD816841F008013E
:100D4000816070470029816802D041F4A00101E070
:100D500021F4A00181607047816841F00401816045
:100D6000704700210160017141718160C160012102
:100D70000174704770B51E4C214694F83800B1F8E4
:100D8000425006281ED9B4F84A10B4F84C00A1EB22
:100D9000000202F10902122A04D8FFF751FB0022D7
:100DA000144B0AE0884204D2FFF74AFB0022124BA0
:100DB00003E0FFF745FB0022104BFFF72AFAFFF78D
:100DC00084FB09E005D12846FFF73AFB0C4A0D4B9E
:100DD000F3E70D4951F82000C5EB45116063B0EB16
:100DE000410F03D9C5EB45104000606370BD0000A2
:100DF0004004002000003440000033400000354033
:100E00006766666666E64B40108A000810B50C4CB3
:100E10002078400713D5FFF7ADFF0A49A08E088060
:100E200008483038018821F010010180001F018836
:100E300041F010010180207820F00400207010BDE6
:100E40004004002040040040F0B416481449446CAB
:100E500008468A6803681448D70542F008050078F8
:100E600022F008064FEA037315D5002B08DB1207A2
:100E700014D408B1082811D1322C0FDA8D6007E0A4
:100E800012070BD508B1082808D1322C06DA8E607B
:100E9000F0BC05F0B3BD002BF2DAE8E7F0BC704718
:100EA0009C02002040010020F306002070B5064699
:100EB0004089204B204C4FF48071002580B362881C
:100EC0007AB1012A0CD1E188491C89B2E1803289CA
:100ED000914205D36580E580FF2801D0401E7081D6
:100EE00070BD70882288904201D9012200E0002262
:100EF000184601F004FA7088B18801442088401C2B
:100F000080B220808142EBD82580A088401C80B22E
:100F1000A080F1888842E3D301206080A58070BD65
:100F2000FFE70022184601F0EAF9A580E580258058
:100F30006580F4E7000C0140B0050020FEE70000EA
:100F4000FCB505464FF6FF7600200C46ADF8006074
:100F500048F205078DF8040020E000BF15F8010BEA
:100F60008DF8040001A9084602F0DAF8BDF8000087
:100F70009DF8041080EA0120ADF800005FF0000049
:100F8000BDF800100A0402D587EA410101E006EA33
:100F90004101401CADF800100828F1DB641EDDD2D1
:100FA0006946084602F0A6F8BDF80000FCBD000046
:100FB0000246002004E000BF12F8013B1844C0B212
:100FC000491EF9D27047000070B5144A85B01088E8
:100FD0000024134901940094039420460494138838
:100FE00007E00D8B009E35440095CD8B019E354466
:100FF000019515889D42F4D0401CC0B28028EED3E4
:1010000000984111074841808480019841110648A9
:1010100081830183818205B070BD0000FC06002041
:101020009C020020CA050020B804002030B50E49FB
:1010300002880A800C4A4388083A13800B1F808874
:1010400018802024151F2C800020401C80B273289B
:10105000FBD341F21110088044F64800108047F29B
:10106000480018802C8030BD202C0140114944F6E6
:1010700048000880091D46F648000880091D41F215
:10108000111008800B48001F018841F020010180E9
:1010900009480021A0F86410A0F86210A0F86010C0
:1010A000A0F85E10A0F85C10A0F85A100348418127
:1010B00081827047182C01409C02002060000020B3
:1010C000F0B54F4B4F480021DA7A0778802A27F095
:1010D00001057DD31C684C4B02F01F0253F82220FF
:1010E0004A4B14421A6802D042F0200201E022F07A
:1010F0002002474C1A60474E94F800C0464CBCF1A1
:10110000020FB4F9044043D1B3F808C0CCF3C00EC9
:10111000CCF3002CE6453BD03C4D2C3D95F802C06D
:10112000BCF1000F04D0BCF1010F0FD0A97033E067
:101130005FEA025C30D55FEA826C2DD44FF0010C7F
:1011400085F802C027F00405057025E05FEA025C1F
:1011500022D45FEA826C1FD55FEA477C0BD447F04C
:1011600004070770B0F802C0BCF1000F06D0418040
:1011700027F0010707700227AF700DE04480002CB4
:10118000F9DD47F001070770244FFF6A4761F2E776
:1011900005704180318041811C4DC78895F84650CB
:1011A0000FB9002C17DC077BAF4214D1B0F90270E5
:1011B00007F26667BC420EDC194FBF895FEA477CC5
:1011C00009D45FEA877C06D45FEA427C03D500E05D
:1011D00012E0FF0709D007785FEAC77C05D027F047
:1011E00001070770418031804181C4800573500937
:1011F00060F3CB221A60F0BD057041804181F0BDE3
:10120000D005002004090020708E00089C020020F8
:10121000F306002010010020CA0500206000002015
:101220000C0A00202DE9F04796B000240C940D9490
:101230000E940F9472B69048816941F400718161F7
:10124000816941F4806181614FF4004002F016FE33
:101250008A4D00212846FFF737FB00212846FFF77B
:1012600029FB874E00213046FFF724FB854F0021E4
:10127000384600F0BBF901204FF47041401C884211
:10128000FCD32846FFF73CFCB1463046FFF738FC5C
:10129000384600F0B7F94FF46020CDE912048DF81C
:1012A000454001204FF004088DF8440010948DF85B
:1012B000508010A92846FFF7B5FC01231A460521E6
:1012C0002846FFF700FD0123022206212846FFF7EA
:1012D000FAFC0123032207212846FFF7F4FC01232F
:1012E00004220F212846FFF7EEFC384600F08AF969
:1012F000684600F032FA6148634E4C300090CDF8F9
:101300000C80CDE901648020CDE9044040000690C6
:1013100080000790202008904FF44050CDE9090448
:101320006946384600F0FCF901212846FFF7CCFA5F
:101330000121384600F05AF901212846FFF7BAFA90
:1013400047F2305115941598401C15908842FAD3F5
:1013500001212846FFF7F6FCADF82C40A04640F2EC
:10136000DC5A4FF4007420E05046CDF854801599B3
:10137000491C15918142FAD330880D9908440D908B
:1013800070880E9908440E90B0880F9908440F9009
:10139000F0880C9908440C9001212846FFF7D2FCF4
:1013A000BDF82C00401CADF82C00BDF82C00A0426C
:1013B000DAD30D98354A40F3CF1633480A30068306
:1013C0000E9941F3CF1444830F9941F3CF138383D4
:1013D0000C9941F3CF1CA0F804C0ACF5C05C40F2FE
:1013E000C371ACF59B7C8C450ED2A6F5C856363E33
:1013F0008E4209D2A4F5C854363C8C4204D2A3F5DF
:10140000C853363B8B4203D3D18841F48041D1800D
:10141000D188490407D41E49028B21F85C2F428BE6
:101420004A80808B888000212846FFF74DFA0021F2
:10143000384600F0DBF800212846FFF73BFA002190
:101440004C464846FFF736FA0220C102401C88424B
:10145000FCD32846FFF754FB2046FFF751FB3846E4
:1014600000F0D0F8FFF73AFA0A493C20087062B65B
:1014700016B0BDE8F08700000010024000240140D3
:101480000028014008000240160500200C0A002038
:10149000600C0020F0060020F0B5384B394C93F872
:1014A0005650374B042D5B6C1DD0256840F22D46FD
:1014B0005D1B656043F6FB25B3F5FA5F33DDB3F5DD
:1014C000FA4F30DC41F6AD17A3F5FA535F4306EB54
:1014D000A7364FF4B5777B4305EBA31375105B106C
:1014E000C4E9065321E043F6D017102641F2620505
:1014F000BB4218DB44F25067BB420EDAA3F56453DB
:1015000045F24C67D03B5F4306EBA736A66140F639
:101510002476734305EB232303E042F24713A361D0
:10152000194BE36101E0C4E90665A3695360E5690D
:10153000401AD56010604543107C0541106A291897
:101540001162D069814200DD1062116A90698142A6
:1015500001DB084600E01062206211684B43117AFB
:101560000B4108411918B2F91400884204DBB2F9A2
:101570001200884200DC08B2F0BD000060000020CC
:10158000400100201401002085EB010010B54FF44C
:101590000054204600F0ACF8002813D00A4908781F
:1015A00040F008000870204600F014F800210748B9
:1015B00000F01CF80648C17E012903D10021C17644
:1015C0000121017710BD00006A060020440002409E
:1015D000040B0020C10002D502490860704702498F
:1015E000486070470404024000000240002901687E
:1015F00002D041F0010102E04FF6FE72114001609D
:101600007047000001684FF6FE7211400160002132
:10161000016041608160C1603149314A08399042BE
:1016200003D1486840F00F0006E02D4A1432904282
:1016300004D1486840F0F00048607047284A2832DA
:10164000904203D1486840F47060F5E7244A3C3288
:10165000904203D1486840F47040EDE7204A503290
:10166000904203D1486840F47020E5E71C4A643298
:10167000904203D1486840F47000DDE7184A7832A0
:10168000904203D1486840F07060D5E7154A111FB9
:10169000904203D1086840F00F0006E0114A14326E
:1016A000904204D1086840F0F000086070470D4A8D
:1016B0002832904203D1086840F47060F5E7094A87
:1016C0003C32904203D1086840F47040EDE7054A8F
:1016D00050329042EAD1086840F47020E5E70000FB
:1016E0000800024008040240406880B270470000D1
:1016F00001460020CA0001D5034A00E0034A1268EF
:101700000A4200D00120704700040240000002405D
:10171000002A026801D00A4300E08A430260704751
:1017200030B5036847F6F07293430C6A8A68224327
:10173000D1E904452C4322438C692243CC692243DE
:101740004C6A22438C6A22431A430260CA68426090
:101750000A6882604968C16030BD00210160416053
:101760008160C160016141618161C1610162416269
:101770008162704710B5114C8CB000212046FFF7F4
:1017800035FF2046FFF73EFF0D4800900D48002131
:10179000CDE901016420CDE903018020CDE90501F7
:1017A0000791089109910A9169462046FFF7B8FF11
:1017B00001212046FFF71AFF0CB010BD580002406F
:1017C000043801408807002010B501218CB008467C
:1017D00002F05EFB1E4C00212046FFF707FF20466B
:1017E000FFF710FF1B4800901B48019000211020BC
:1017F000CDE902018020CDE90410069107910891FE
:1018000009910A9169462046FFF78AFF01220221C9
:101810002046FFF77DFF01218DF82F1004208DF861
:101820002D008DF82E100E208DF82C000BA802F044
:1018300013F80F208DF82C000BA802F00DF80121F1
:101840002046FFF7D3FEFFF795FF0CB010BD000058
:1018500044000240043801402407002030B540F61F
:10186000AA21204AC184838B1488E31A9BB20F2BD0
:1018700010D312888283037E002253B11A4BB3F92E
:101880000A30062B05DB194B1B78022B03D0002BEB
:1018900000D1828430BD164B40F68B255B6CA3F2E1
:1018A0002D14AC420FD2428B521C92B24283642A56
:1018B000F0D364224283B0F924208A4201DA02EB99
:1018C0002111818430BD41F29414A342FADBB0F9B6
:1018D0002430002B02DDA3EB211100E000218184E4
:1018E000428330BDFC06002060000020F30600208B
:1018F0004001002010B50446B0F9020043F69911EA
:1019000048438113E06840F26662504301EBA03027
:10191000E060B4F9001043F6991251438A1321692B
:1019200040F26663594302EBA131216104F0E4FC0B
:101930006061A18840F6AB2208444010A0F5154133
:101940005539E062914205D9A0F5F851FF39521C92
:1019500091421DD249F25451884202DDA0F5204047
:1019600002E0A0F5F850FF38206300EB400040F3A0
:101970004F002085B4F924104A42904201DA104603
:1019800002E0884200DD0846E083228461848AE028
:10199000A0F5FE42FF3A41F255518A4214D8A2F610
:1019A000AA20206300EB400040F34F002085B4F9EB
:1019B00024205142E183884201DA084602E0904245
:1019C00000DD1046404250E0A0F5D442AA3A8A42D7
:1019D00015D2A2F6AA20206300EB400040F34F018D
:1019E0002185B4F924004242E2832084914201DA45
:1019F000104602E0814200DC0846608453E0A0F516
:101A0000AA42543A41F256539A4215D2A2F6AB205A
:101A1000206300EB400040F34F002085B4F9241010
:101A20004A42904201DA104602E0884200DD084650
:101A30004042E083218419E0A0F5804241F25453F2
:101A40009A4215D2A2F6AA20206300EB400040F390
:101A50004F012185B4F92400E0834242914201DA2A
:101A6000104602E0814200DC0846208462841AE0CD
:101A7000A0F52852AB3A8A4215D2A2F6AA202063DA
:101A800000EB400040F34F012185B4F92400E083CE
:101A900042422284914201DA104602E0814200DC97
:101AA00008464042A9E7B4F91E006FF4BF714843ED
:101AB0008013E080B4F92000484380132081B4F9FA
:101AC000220048438013608110BD70471548164AB4
:101AD0004FF480410078042821D002F13C03D08AE1
:101AE0009B88C01A00B22F2801DD001108E00028F1
:101AF00001DD002007E00D4B984201DA184602E0B4
:101B0000402800DD40209389184400B2884203DC5D
:101B100040F26661884200DA084690817047918100
:101B200070470000F3060020B8040020C0FEFFFF4D
:101B300038B54B484B4902880B889A1A92B20F2A43
:101B400071D30988484C01804FF0FF01E2884FF4BF
:101B50007A7355044FF4967002D51622009103E073
:101B6000950403D515220091014670E0D50402D5F5
:101B700014220091F8E7150502D513220091F3E72E
:101B8000550502D512220091EEE7950502D51122E6
:101B90000091E9E7D50502D510220091E4E715068A
:101BA00002D50F220091DFE7550602D50E220091E3
:101BB000DAE7950602D50D220091D5E7D50602D5C4
:101BC0000C220091D0E7150702D50B220091CBE73C
:101BD000550702D50A220091C6E7950702D50922CA
:101BE0000091C1E7D20702D008220091BCE7228908
:101BF000550702D507220091B6E7950702D50622C0
:101C00000091B1E7D20702D005220091ACE7A27A99
:101C1000D20702D004220091A6E7A289D40603D5F8
:101C200003220091A0E719E0140702D502220091D7
:101C30009AE7540703D4940701D4D20702D00122B3
:101C4000009191E70020034602460146009002F011
:101C50002BFEBDE838400248FFF728B938BD000028
:101C6000000A0020FC0600200C0A0020F0B55948AC
:101C7000594982880B889A1A92B29C2A64D309889F
:101C8000818056490A880146002A0B7843F00201F8
:101C900056D11646524A1C0715680246127822F0A1
:101CA000020274D54F4C0746E4887F785FEA845C73
:101CB00002D547F0010701E027F001074770A704AC
:101CC000477802D547F0020701E027F00207477086
:101CD000670401D4E70703D0477847F00807477047
:101CE000640603D5447844F0040404E01C0603D4DD
:101CF000447824F004044470EC0450D4354C9A0722
:101D0000247824F0100423D4324D42782F7A2D7891
:101D1000012A45F0100514D0022A16D02D4C042AB1
:101D2000A47804F1010C0CF0FF0C13D0072A25D085
:101D3000032A23D0052A21D0062A1FD021F0100122
:101D400042E0B90702E00570F0BD39070029FADB6F
:101D50000470F0BDFA0601D41A060AD50170022CEF
:101D600004D280F802C0BCF1020FF2D341F080012E
:101D70002AE021F0100101708670F0BD877A7F069D
:101D8000F7D5032C04D8017080F802C0F0BD0FE035
:101D90005107D8D51906D6D443F0800114E002705B
:101DA0004178CB0701D18907F0D522F010010BE073
:101DB000E9040BD49907E9D4818AC82902D2491CC5
:101DC0008182E3E743F00A010170DFE70270868257
:101DD000DCE70000D4060020FC060020FE06002000
:101DE0009C0200200C0A0020094944F648000880A3
:101DF000091D46F648000880091D41F6CC400880C0
:101E00000348001F018841F0200101807047000055
:101E1000182C0140084946F668000880091D088012
:101E2000091D41F2555008800348001F018841F008
:101E30002001018070470000182C014010B5C288B5
:101E400000210AB1032206E002890AB1022202E05F
:101E5000428912B10122027000E0017004784FF44F
:101E6000804344F6206244B1012C06D0022C07D0F6
:101E7000032C01D14180818010BD4380828010BD40
:101E800041F23331418040F6B731F4E730B5CD8DC2
:101E900000230B240522854202DCB1F92C0030BD61
:101EA0004D88854202DBB1F9000030BD01EB8205AF
:101EB0006D88854201DD144601E013DA134604EB18
:101EC00003024FEA52029A42F0D101EB830231F849
:101ED000231054889288521A001B424301EB62205F
:101EE00000B230BD31F9220030BD0000054920B1FB
:101EF000086940F080000861704703484860034863
:101F0000486070470020024023016745AB89EFCD50
:101F100006494FF47A70CA68D20705D0401E000403
:101F2000000CF8D1FF2070470020704700200240CD
:101F300011480321A0F14C0280F836100021518194
:101F40000E4A1186D162D1831184518481620C4979
:101F50008A6CB2F5206F01DBA3228262897A11B10B
:101F6000816A49428162C16A41F3910181628803B9
:101F7000044908627047000060000020200500202E
:101F800040010020680800200449002048810881A1
:101F9000C862886202490862704700006000002041
:101FA0008C080020F0B53B4988894A89801A80B2A4
:101FB0000F2866D388894881CA8937480B3A272A6F
:101FC00026D28A7822BB8268364B42F480728260C5
:101FD000324A354C354D12785607314A0AD4344EC0
:101FE00036881680334A12881A80334A1288228033
:101FF000324A09E0324E36881680324A12881A80F8
:10200000314A12882280314A12882A8001228A703D
:102010002F4B304D19469A7F0968802A32D302F03F
:102020001F0255F8222011422CD0826822F480121F
:10203000184E8260123614461215B778521C62F39D
:102040008617254AB77093F816C01778BCF1800F31
:1020500027F0020608D30CF01F0C55F82CC011EA2B
:102060000C0F01D147F0020616701A7E802A0DD39C
:1020700002F01F0255F82220114207D144F400213A
:102080008160F0BD826842F48012D1E724F400211F
:10209000F6E70000F00600209C020020400100202E
:1020A000B0040020B2040020B4040020B6040020D4
:1020B000A0040020A2040020A4040020A604002004
:1020C000A8040020AA040020AC040020AE040020D4
:1020D000D0050020708E0008B804002070B520489C
:1020E00081890289891A89B20F292FD381890181B7
:1020F0001C4B1D4819465D7A06681C4C096846F061
:102100000402802D07D305F01F0554F825502942FD
:1021100001D126F0040202609A7B802A17D302F0D4
:102120001F0254F82220114211D1026822F002024B
:102130000260DA7A802A0ED302F01F0254F82220BD
:10214000114208D1016821F00801016070BD0268E8
:1021500042F00202ECE7016841F00801F5E70000F7
:10216000F0060020D00500209C020020708E0008A0
:10217000F0B51D4C1B4A4FF0010C94F83B5094F8FD
:102180000AE0144692F83C3094F838402B43651C22
:10219000EEB2154D95F83D700025BEF1FF0F0AD047
:1021A000BEF1000F06D18B4213D155700C2C01D219
:1021B00082F83860F0BD834202D182F801C0F5E7B1
:1021C0008B42F7D15570B80709E000BF82F838504C
:1021D000F0BD8342FCD1F84382F801C0800700289B
:1021E000F4D0F0BD4004002040010020F0B5CA78D2
:1021F000002502F00F03D20601D58A7813430A782E
:102200004FF00F0E12F0FF0F4FF001021CD00468C8
:102210000F8802FA05F63740B74211D14FEA850C14
:102220000EFA0CF724EA070703FA0CF43C43CF78C4
:10223000282F02D0482F02D002E0466100E006615C
:102240006D1C082DE4D304600C88FF2C1ED9446853
:102250005FF0000606F1080702FA07F50F882F4025
:10226000AF420FD14FEA860C0EFA0CF7BC4303FACB
:102270000CF73C43CF78282F00D14561CF78482F09
:1022800000D10561761C082EE4D34460F0BD000047
:10229000F0B5144C002801DAE36900E06368420DF0
:1022A000120185B2C0F301579540C0F30346032FD6
:1022B00005D0C2020AD50322B240934307E023F0BF
:1022C0007062636823F07063636002E0AB4343F0C5
:1022D000706201B12A43002801DAE261F0BD626058
:1022E000F0BD0000000001400246002092680A4252
:1022F00000D00120704741617047016170470AB109
:1023000001617047416170470F4A104B92F83810D5
:102310005B5C834201D1012004E00D4B5B5C834296
:1023200003D1002082F83A0070470A4B5B5C83427D
:1023300001D18120F6E7084B595C814201D1802010
:10234000F0E70320EEE70000400100203092000893
:102350004292000836920008489200080A4810B5D8
:1023600001784FF000024C0708494FF0FF038968DD
:102370004FEA017105D5002901DA827210BD83721E
:1023800010BD0029FBDBF8E7400100209C02002083
:10239000F0B5194E194C0022E31CA6F1060CB75CEF
:1023A000A518ED78FF5C0D430F43BD421FD01CF80C
:1023B0000270FF5C0F43BD4219D015460023A618DA
:1023C000F6780E43C6545B1C1CF80220DBB2062BC9
:1023D000F5D3C17881700179C17000214218491C80
:1023E00015711CF80550C9B20629F7D3F0BD521C6F
:1023F000D2B2032AD3D3F0BD028A000840040020E1
:1024000010B502460021064B06205C186478944201
:1024100000D10846491CC9B20629F6D310BD0000F8
:1024200040010020214810B590F867100022204894
:10243000012936D11F49898899BB1F491E4B4C6C15
:1024400040F6B831B3F86E308C4227DD1B4909786D
:1024500021BB90F82711491CC9B280F82711C8295F
:102460001CD380F827210146D0F82C4191F828117F
:10247000A34203DD052908D2491C01E041B1491EF0
:1024800080F82811C9B2052902D3012180F826114C
:10249000191B074C2C3C6162C0F82C31B3F5FA6F64
:1024A00003D280F8262180F8282110BD600C00207E
:1024B0009C020020CA05002040010020F3060020F5
:1024C0004FF4C0428260002141620E22828141F2BB
:1024D00062020261082282824FF46042C28201835A
:1024E0004FF07842C0E9072140F6C41101807047DF
:1024F000B0F90010B0F90220891A41600269037D29
:102500004A431A41436A13444362026A934200DD1C
:102510004262436AC269934200DA42628268436A55
:102520004A43017B0A410B41D118B0F918208A4275
:1025300001DA10467047B0F916008842FADC08B29A
:102540007047000010B514481449B0F88C200B886F
:102550009A1A92B2B2F5437F1DD90988A0F88C105F
:10256000B0F88A1020F8581F002242860C480D4C03
:10257000C2888280C180C38983812489891AA4B2D8
:10258000C4818160E11A0161074A818AC182928A0D
:102590008282511A816110BD40010020FC0600209A
:1025A000280C0020200500206000002009480A496E
:1025B000B0F8AA200B889A1A92B241F684639A4224
:1025C00006D3098820F8AA1F418881800021418014
:1025D0007047000040010020FC0600200D480178F3
:1025E000C90702D00C49098801E04FF6FA71C165AC
:1025F000094901201039088007482438018841F032
:102600000101018004481838018821F01801018077
:102610007047000040010020240400400A49D1F81E
:10262000902012B1521EC1F8902031F88A2F521C0E
:1026300021F81A294A6A521C4A628A8F521C8A87D8
:1026400001F8380C70470000400100201CB52D48EF
:1026500090F83B3090F83C20934252D000248DF803
:10266000044053408DF800309DF800300122012BCA
:1026700008D09DF80030022B09D09DF80030042BC3
:102680000AD00DE01F498DF80420443108E01D49AF
:102690008DF80420463103E01A498DF804204831B2
:1026A0009DF80420012A2CD190F83D309DF800407F
:1026B000154AA34217D090F83E309DF800402342BF
:1026C00008D0B0F84C30A0F84A300B881488E31AD0
:1026D000A0F84C3090F838302BB1B0F84030148866
:1026E000E31AA0F8423012880A80A0F8402010F8BF
:1026F0003E1F9DF80020114300F801199DF80010BD
:1027000001701CBD40040020FC06002070B5344D53
:1027100040212846FFF7E8FD840080212846FFF786
:10272000E3FD44EA4004A9152846FFF7DDFD044314
:10273000E1B22C4C94F870508D4250D04D4084F84A
:102740007010012D03D0022D01D0042D47D194F833
:102750007400A84384F8740094F87320AA420FD040
:1027600084F8735094F8722001238B401A4207D1E9
:102770001A4384F8722094F87110491C84F871107F
:1027800094F87110042928D330B1012811D00228FF
:102790000FD004280DD012E01348C18821F0400169
:1027A000C1802078002184F83B1020F06000207068
:1027B00005E0217841F02001217084F83B000B49AD
:1027C00094F83B0091F82720904204D081F827002C
:1027D00007492020087000F00DF884F84C5070BDB7
:1027E00000100140400100200C0A0020600C002075
:1027F000F006002070B50D4D40212846FFF774FD0E
:10280000840080212846FFF76FFD44EA4004A915A3
:102810002846FFF769FD04430548072100F8704F7B
:102820000171002141708170C17070BD00100140C4
:102830004001002070B5344890F83A10CA4392071E
:1028400061D001F0030280F8392090F83D305B063A
:102850001B0E80F83D30012A01D0812A02D15B1C79
:1028600080F83D300278D2074DD0DBB203F0010290
:10287000C3F34004A24246D1B0F84E400025641C88
:10288000A0F84E40204CA0F8505090F83E60A47A3A
:10289000B24202D080F83E200DE0A607B6EB837F5F
:1028A00002D080F83F5006E090F83F30642B02D20F
:1028B0005B1C80F83F3090F84030642B0CD25B1CDE
:1028C000DBB280F84030022B06D204F001039342C1
:1028D00002D1022280F84020012901D0002912D122
:1028E00090F83820C16D00EB820291610163D0E95C
:1028F00006121144D0E908231A441144826A114493
:10290000C26A1144416370BD40010020FEE700002F
:102910002DE9F04F00BF00209E4E9F4AA6F5127190
:10292000A6F5BE79A6F1440B06F1440E804601F5EA
:10293000E074A1F1780301F5457A1D5C15F0C0073C
:1029400006D0402F51D0C02F77D0802F76D004E111
:1029500015F01F0504D0154440F080072F7201E0E8
:1029600082F80880012826D0022824D0032822D00B
:10297000042820D008281ED010281CD0874D55F8D8
:1029800020C0DCF8005054F820703D40CCF80050D6
:10299000824D55F820C0DCF8005056F820703D43B9
:1029A000CCF800501D5CAD0659F820502F6813D5A7
:1029B0003AF810C03EE051F820502F6854F820C07B
:1029C00007EA0C072F6051F820502F6856F820C0F6
:1029D00047EA0C072F60E5E7DFF8B8C10CF1F00C0F
:1029E0005CF820C007EA0C077EE015F01F0504D054
:1029F000154440F080072F7201E082F8088001281A
:102A00001DD002281BD0032819D0042817D008286D
:102A100015D0102813D0614D55F820502F6854F868
:102A200020C007EA0C072F605C4D55F820502F6836
:102A30005BF820C047EA0C0756E00BE056E051F87F
:102A400020502F6854F820C007EA0C072F6051F877
:102A50002050ECE715F01F0505D0154440F0800725
:102A600085F8217001E082F82180012825D0022814
:102A700023D0032821D004281FD008281DD01028D7
:102A80001BD0464D55F820C0DCF8005054F820709B
:102A90003D40CCF80050414D55F820C0DCF80050C6
:102AA0005EF820703D43CCF800501D5CAD0615D596
:102AB0003A4D3AF81070CC3514E051F820502F6898
:102AC00054F820C007EA0C072F6051F820502F68F7
:102AD0005EF820C047EA0C072F60E6E72D4D3AF874
:102AE0001070E03D55F820502F6036E015F01F05BE
:102AF00005D0154440F0800785F8217001E082F888
:102B00002180012830D002282ED003282CD0042880
:102B10002AD0082828D0102826D0204D55F820C0CB
:102B2000DCF8005054F820703D40CCF800501B4DAC
:102B300055F820C0DCF80050164F883757F8207041
:102B40003D43CCF800501D5CAD06B1D4114F3AF8AE
:102B50001050E03F57F820703D60401CC0B2112873
:102B6000FFF4EBAEBDE8F08F51F820502F6854F819
:102B700020C007EA0C072F6051F820502F68DFF8BB
:102B800014C00CF1880C5CF820C047EA0C072F60D9
:102B9000D9E70000FC900008D0050020F88E00085E
:102BA0004FF40771C1824FF45861018340F614510C
:102BB00081837047F0B5C48AB0F900608681B0F9AE
:102BC0000250C581B0F9043002270021012203829E
:102BD000AB4204DBB54202DDC78042810CE0B34268
:102BE00004DBAE4202DDC78041811CE09D4205DB73
:102BF000B34203DDC2804781018115E0B54204DBA9
:102C00009E4202DDC280418105E0AE4205DB9D426D
:102C100003DDC1804281078106E09E4204DBAB42B6
:102C200002DDC18047810281C388458900EB4307EB
:102C300000EB4505BB89AE899B1B0FFA83FEA0F80C
:102C400012E00689AB8900EB460CBCF80CC0A3EB84
:102C50000C038382B0F91830B7F90CC0A3EB0C0C4D
:102C6000B4EB4C0F04DA80F82010A3F1A10113E0BB
:102C7000A64503DD80F82010B9890BE026B1012EAE
:102C800004D0022E10D004E0062100E0052180F8D7
:102C90002010A989091B6D31418309B2B1F5586F24
:102CA00004DB5B1E438304E00421F0E7002900DC21
:102CB0004283418B8183F0BD0B49002288760A62F2
:102CC000CA614A62094A32F9103002EB40028B6253
:102CD000B2F90220CA62064A32F810000882A1F84E
:102CE0006000A1F862007047F00100205A920008CD
:102CF0004E9200082DE9F05FF048F14982880B8878
:102D00009A1A92B20F2A44D3098881468180ED48ED
:102D10000127ED4C0188ED4E002579B3491E018055
:102D2000E573EB49A5622068B1F90210430742F64A
:102D3000AA2218D4F38843F40053F380E44B1B78A1
:102D40009B0709D5A36823F08003A360A4F87C50F7
:102D500084F87E5084F87F50C30404D484F8F07063
:102D6000C4F8EC5003E084F8F050430707D49142D4
:102D700005DB84F8F470A4F8F25004E010E084F865
:102D8000F450430703D4914201DBC00703D084F819
:102D90001151BDE8F09F84F81171A4F81251F8E7C1
:102DA000B4F8180143F69821884202D2401CA4F8D6
:102DB000180101F08FFDDFF81C83DFF800B398F8ED
:102DC0005000ABF1180B10B1FEF77AF905E09BF853
:102DD000001021F001018BF80010FFF723FB00F039
:102DE000B5F9BD4841F26801426C4FF400608A4277
:102DF00001DBBA4904E0B2F57A6F02DAB749091D7E
:102E0000086098F85100DFF8C0A2B54BDFF8D48213
:102E1000C007AAF12C0A2ED0987B802827D32078CF
:102E2000800724D4E07B8AF80500A948514603783E
:102E300023F002030370ABF80250CBF814509BF858
:102E4000003023F001038BF80030B079400609D43C
:102E500040F63C70824201DD0020FBE008208AF849
:102E60000370F7E0CD700020AAF80A50F2E08AF86B
:102E70000350AAF80A50A068020501D50820E9E02D
:102E8000944991F83F20D10743D0E17B8AF805109F
:102E90009E465B7A802B47D323785B0732D4F38836
:102EA0009B0403D520F02000A06032E0ABF8025074
:102EB000CBF814509BF800C040F020002CF0010C1F
:102EC0008BF800C0A0609EF8170080280BD300F09C
:102ED0007F0C4FF00040DEF8003020FA0CF0034287
:102EE00001D1277100E025712079C00701D1900739
:102EF00005D50320032901D08AF80870AAE0002034
:102F0000A562A7E020F02000A060F08820F4005027
:102F1000F08094F8260101280BD06E4890F86300E9
:102F200048B1FDF791FF0FE0216841F004012160F5
:102F3000B8E709208EE0A068C10502D520F008009E
:102F400001E040F00800A06094F8462043F23330DE
:102F50004FF480477AB143F69911012A1ED0032A13
:102F600098F800206048C2F381021AD0012A30D0BC
:102F7000022A2ED02AE098F80010C1F3810101291D
:102F800009D0022907D043F2AE71A4F8141100BF92
:102F9000A4F8440021E0A4F81401F9E7A4F814010E
:102FA00019E0012A0BD0022A09D090F85600042813
:102FB0000CD0A4F8147100BFA4F844700DE0A4F87C
:102FC000147190F85600042805D0F5E7A4F81471A0
:102FD00001E0A4F81471A4F84410FEF771F89BF80E
:102FE0000010C90702D0BBF8021001E03848818800
:102FF000A9F8121008B2B4F944104843C0F38F3155
:103000005046AAF81210B94200D9478237490978C8
:10301000C90605D5428A41F233318A4200D2418243
:103020002189C1F3C002C1F300218A4205D1428A3D
:1030300040F6CC418A4200D94182B17AC90700D01A
:103040004582BAF81200A06200287FF705AF284831
:103050000570022099F81A1099B9022824D080B17D
:103060001D4A11788D0608D5B5796D0605D51F4D19
:103070002D78ED0965F386111170F18821F40A614C
:10308000F1801549496C4E290ADBF1880A0607D5FB
:1030900021F08001F1800E490A7822F002020A70C4
:1030A00089F81A00E07374E6B8F83820002AD7D1FE
:1030B00043F69822A8F83820D2E700001C09002027
:1030C000FC060020FE0600209C0200200C0A0020C6
:1030D000CA050020600C002040010020100C0140B7
:1030E000D0050020B804002060000020D406002095
:1030F0001007002070B500230C8863F30F02012530
:1031000005FA03F6344206D0C3F10F0605FA06F1BC
:10311000114361F30F025B1C102BF1DB028070BDC9
:1031200070B500230C7863F30702012505FA03F656
:10313000344206D0C3F1070605FA06F1114361F3E4
:1031400007025B1C082BF1DB027070BDF0B51F4855
:1031500090F866301E48012B816821F4006232D15C
:103160001C4BDE8874062ED41B4D0F054FF0000457
:10317000B5F902501ED4194A526C642A11DC40F68B
:10318000386295420DDAB2040BD4027852070ED49D
:10319000B0F8D42040F6B835AA4203D2521CA0F8A9
:1031A000D420F0BD41F4006181605C81F0BDA0F8E5
:1031B000D440F0BD41F2CD018D42FADD997AC907C4
:1031C000F7D18260F3E78260F0BD0000600C002060
:1031D0009C0200200C0A0020CA05002040010020AB
:1031E000F0B5364D364F044695F83B0097F83B1046
:1031F00023780843EE1C6278834205D1E0781146BB
:10320000FEF7B6FF207908E094F802C084450CD19F
:10321000E1781046FEF7ACFFE07905F82F0F28782B
:10322000805D6870287BE877F0BD82421DD16146E1
:103230001846FEF79DFF95F84E1095F83B00814229
:1032400007D1B97A09B1A17900E0617985F82F1029
:103250001EE06978012901D0A17922E0617927E097
:10326000297841F00401297012E0E1788142DBD134
:1032700019466046FEF77CFF95F84E1095F83B0026
:1032800081420AD1B97A09B1617ADFE7217ADDE7B3
:1032900015F82F1F895D6970C5E76978012906D087
:1032A000617A85F82F10B97A0029F1D1D8E7217A0F
:1032B00085F82F10B97A0029EAD0D1E74004002020
:1032C000400100200B48017821F0020100F8381B72
:1032D000002100F8181941778177332181854185D4
:1032E00008214184012100F81F1C034880F839108F
:1032F0007047000040040020400100200D4900B547
:103300000B4851F8012F40F8032F89888180084825
:1033100001210930FFF73CF8054802211330FFF77F
:1033200037F8034804211D305DF804EBFFF730B88F
:103330004004002040010020094944F6480008806C
:10334000091D46F648000880091D41F21110088049
:103350000348001F018841F02001018070470000F0
:10336000182C01402DE9F047664C674B0025A078EA
:103370000126654A103305287ED2DFE800F00313EA
:10338000113E1100108820F0010010801D805F4860
:103390000580001F0580001F0580FFF7CDFFA67088
:1033A000BDE8F087594941F244401C39088057492B
:1033B00045F6580024390880091D47F25800088056
:1033C00052492020283908800020401CC0B27328B0
:1033D000FBD3FFF7B1FF4C4984F85C502C3147F622
:1033E000906008804848143006801D80108840F0A6
:1033F000010010800220A070D2E700215FF00100E0
:1034000004EB410204EB4003B2F85020B3F8503013
:103410009A4200D20146401CC0B20628F0D33C4874
:10342000405C84F83900FFF74DFF1D2000F0F3F9F0
:1034300000F076F8374E38484FF4807996F83B1014
:10344000012904D002291BD0042930D047E04021B3
:103450008046FEF749FF870080214046FEF744FF83
:1034600047EA400749464046FEF73EFF074347F01C
:10347000010084F83B0000E03DE0224809302CE0E8
:1034800040218046FEF730FF870080214046FEF74E
:103490002BFF47EA400749464046FEF725FF074312
:1034A00047F0020084F83B001648133015E0402135
:1034B0008046FEF719FF870080214046FEF714FF83
:1034C00047EA400749464046FEF70EFF074347F0EC
:1034D000040084F83B000B481D3002F0DBFD94F83B
:1034E0002F0086F838001D2000F0ABF90420A070F2
:1034F0000A48057054E7108820F0010010801D80F4
:10350000A5704DE740040020000800403C2C01401D
:10351000088A00084001002000100140F306002046
:103520002DE9F041344C14F82F0F344DE072402156
:103530002846FEF7D9FE860080212846FEF7D4FEF5
:1035400046EA4006AF1539462846FEF7CDFE06434B
:10355000207BF1B22F3C814215D084F83C00402101
:103560002846FEF7C1FE860080212846FEF7BCFEF5
:1035700046EA400639462846FEF7B6FE064384F87A
:103580003B60FFF763F81E4D95F83B00012827D0FC
:10359000022828D0042829D0174894F83B10273057
:1035A000085C04F8300F14F80109FEF729FF04F84D
:1035B0002F09A87A00B10120607001F017FA94F881
:1035C0004E0094F83B10884206D094F83800062844
:1035D00002D2401C84F8380084F84E10BDE8F08117
:1035E0000548093004E00448133001E002481D306A
:1035F000BDE8F041FFF7F4BD400400200010014099
:10360000400100202DE9F041524991F87200AA28AA
:103610007ED191F8730055287AD14F4C00200A5C76
:103620002254401CC0B27428F9D34C4E2069C6F80D
:103630000100A08AA6F80500D4F81600F060D4F8BE
:103640001A003061D4F81E001234706102F0C8FC18
:103650004349608A888102F0DDFC207D123CC0076E
:10366000307802D040F0040001E020F004003D4931
:1036700030704FF480403C4D886114F8280F85F875
:103680002000608B6880A08BA880E08BE880208C75
:103690002881608C354F688194F8240087F8D20027
:1036A00014F8011C304686F83B100026C0F89460E0
:1036B000FFF724FE2E48A18E0183E18E4183218FE6
:1036C000818394F84210283C012908D0022901D0B6
:1036D000032909D0297821F00C01083107E0297865
:1036E00021F00C01091D02E0297841F00C0129703C
:1036F00094F86E20012162B1012A01D0022A0BD078
:1037000087F8461094F864301A4A4BB1518108E0AA
:1037100014E087F84660F5E7022287F84620F1E7D3
:10372000568194F8701001290AD094F86D1051B1A7
:1037300001290BD04FF48051A0F87610BDE8F0813C
:1037400044F21C71F8E74FF40051F5E741F255518E
:10375000F2E7000000FC0008600C0020400100209F
:1037600060000020F80B0020B80400209C0200201C
:10377000200500200C0A00207CB50121082000F063
:10378000ABFB4FF48070ADF8040010248DF80740B7
:1037900001208DF8060001A91548FEF727FD01213B
:1037A000092000F099FB01211248FEF771FD082065
:1037B000ADF8000004208DF803000F4E03258DF8AE
:1037C000025069463046FEF711FD08213046FEF7EB
:1037D00092FDADF800408DF803408DF80250694627
:1037E0003046FEF703FD10213046FEF784FD7CBD18
:1037F0000014014000023000000C0140FEE7704759
:1038000000F01F02012191404009800000F1E020FA
:10381000C0F88011704700F01F020121914040095B
:10382000800000F1E020C0F88011704700F01F0216
:10383000012191404009800000F1E020C0F8001112
:10384000704700F01F02012191404009800000F103
:10385000E020C0F80011704770B50F23C4780178DC
:103860000122F4B1144C2468457804F4E064C4F5F2
:10387000E064240AC4F10406E3408478B5401C40A7
:103880002C4301F1E021230181F80034007800F09D
:103890001F018A404009800000F1E020C0F80021AB
:1038A00070BD01F01F0082404809800000F1E02057
:1038B000C0F8802170BD00000CED00E00249084313
:1038C00002490860704700000000FA050CED00E0B6
:1038D0002DE9F05F00261D20FFF792FF6C4CDFF80A
:1038E000B4B1A4F1B000A77E90F83810DFF8A8E1D9
:1038F000DFF8A8A100258F427ED0E776A176626A24
:10390000036B5A434FEA12499BF80820120702D56D
:103910001EF8012000E00A4694F812C0BCF1010F25
:1039200009D004EB4206B6F902C0C4F828C0B6F9C3
:103930000460E6620CE043F6FF7CC4E90A5C90F8A0
:103940003DC05FEACC7C01D012B102E0052A00D173
:10395000012600EB47074FF0804CBF893F04B7FBBF
:10396000F3F3E361476BBCFBF7F7276294F813C0EE
:10397000BCF1000F06D0BCF1010F05D03B4403EBB6
:10398000D3735B10636201E03B466762DFF810C1EE
:103990004FF6FF7707EA8307ACF808709AF80070D3
:1039A00090F80A8090F83DC0082F08F003070CF04B
:1039B000030C05D067450BD1B8F1000F05D008E026
:1039C000674505D0B8F1000F03D05B42636200E0A9
:1039D0006562C6B1636A002B03D006DD228D05E067
:1039E0000AE0304B33F8122000E0A28DA4F86020EA
:1039F000227822F0200222709AF80020042A07D0B0
:103A0000082A05D012E0B4F8603003EB0902EDE7B4
:103A100080F8405065629BF80800000701D51EF849
:103A20000110204830F81100A4F860001E49606AB7
:103A300009883E314843B4F8601001EB204006B2DB
:103A40001D20FFF7F3FE606A002807D021784FEAB7
:103A500081600ADD002804DAA08D09E0B4F8600076
:103A600006E0E06AB04208DB0CE0002802DA208DB4
:103A7000208208E0A06AB04204DD208241F02000EC
:103A8000207000E02682257565752586BDE8F09FCB
:103A9000F00100209C0200203C920008F306002068
:103AA000E40900204E9200082404004043184FF41B
:103AB0008042934210DD904202DD104600210BE06F
:103AC000914202DD0020114606E08003B0FBF3F0D6
:103AD00000B2C0F5804109B241EA004070470000E1
:103AE0002DE9F043002340F2AE440E25446003620A
:103AF000058144F24C260827C6600782DFF834901F
:103B000043F6FF7CA0F81290A0F814C04FF0704864
:103B10004FEA8C32C0E906824C600B620D81CE60A8
:103B20000F82A1F81290A1F814C0C1E90682BDE885
:103B3000F083000000C0FFFF00214162094981605D
:103B40000E2181814FF6BF510161082181824FF41E
:103B50004041C18243F6FF7101830907C1610249F7
:103B600001627047638A010000C0FF0F064941F6F9
:103B7000A260088005480168054A01F4E06111432C
:103B80000160BFF34F8FFEE7442C01400CED00E0D5
:103B90000400FA0538B501210D2000F09DF94FF41D
:103BA000E060ADF8000018248DF8034003258DF87F
:103BB000025069460D48FEF719FB4FF46040ADF81E
:103BC00000008DF803400A4C8DF8025069462046EB
:103BD000FEF70CFBA014ADF8000048208DF80300A0
:103BE00069462046FEF702FB38BD00000008014090
:103BF000000C0140F0B50121CE028DB0304600F03E
:103C00006BF9594F384601F063FB08A801F08CFDB1
:103C10004FF45860ADF824000024ADF82040202077
:103C2000ADF82200ADF8264008A9384601F02EFD77
:103C30000021384601F081FD4FF6FF71384601F052
:103C400086FD01220021384601F012FD012138468F
:103C500001F0FAFA04A801F012FBADF81060701040
:103C6000ADF81200ADF81440A220ADF816007000B7
:103C7000ADF81800ADF81A40ADF81C4004A938465C
:103C800001F0ECFA6025ADF80050ADF80440ADF855
:103C90000840ADF80C40ADF80240ADF80640ADF874
:103CA0000A40ADF80E406946384601F0D1FB69463E
:103CB000384601F013FC6946384601F059FCADF86E
:103CC00000500125ADF8045040F61450ADF8060040
:103CD000ADF80840ADF80C40ADF80250ADF80A4020
:103CE000ADF80E406946384601F086FC01213846A1
:103CF00001F0CEFA0821384601F0EAFB3146384699
:103D000001F02CFC0821384601F070FC31463846A1
:103D100001F0A4FC7021384601F0ADFC18208DF8AC
:103D20002C008DF82D408DF82E408DF82F500BA8CB
:103D3000FFF792FD0C480C30018841F080010180B2
:103D400009481430018841F001010180001F0480FE
:103D50000121384601F0A6FA8DF828500121384695
:103D600001F0AAFA0DB0F0BD002C01407047000030
:103D700070B50189C1EB411101EB4101CA0B4281D0
:103D80000B49104603F008FD09480C38B0F90C2027
:103D90000168B0F90E4001FB02F54368614303FB83
:103DA000145503FB0211AD138913C0E9055170BD11
:103DB000F009002040F21341416008218160862112
:103DC000C1604FF4804101614942416100210162BB
:103DD000C16270470162704710B501884288891A34
:103DE00009B20183B1F5005F02DBA1F5804104E077
:103DF00011F5005F02DC01F580410183B0F9182064
:103E000041685143C1618368846A5343C2681B128D
:103E1000624303EB2222036A1A44114402628A13AA
:103E2000426241698A4203DB01698A4200DC114631
:103E30008A1AC0E90A21028E4FF40373594302EB38
:103E4000A13202860B4A1278082A04D10A4AD36E9C
:103E500003EBA131D166B0F93010B1F5804F02DD2E
:103E6000A1F5804103E0002902DA01F580410186D5
:103E700010BD0000F3060020200A0020034A51680C
:103E800021F440410143516070470000001002409E
:103E9000044A0029516901D0014300E08143516186
:103EA0007047000000100240044A0029D16901D087
:103EB000014300E08143D1617047000000100240DF
:103EC000044A0029116901D0014300E081431161D6
:103ED0007047000000100240044A0029916901D097
:103EE000014300E0814391617047000000100240EF
:103EF000044A0029D16801D0014300E08143D16028
:103F0000704700000010024030B524494A6812F0A2
:103F10000C03234A03D0042B01D0082B26D00260C7
:103F20004A680F231F4C03EA1212A35C0268DA40AE
:103F300042604B68072505EA1323E35C22FA03F38A
:103F400083604B6805EAD323E35CDA40C2604B68C8
:103F5000032403F4404104EA933303EB9161114BD2
:103F60001B1F595CB2FBF1F1016130BD4A680E4B79
:103F70001A404B68140103F4803303D5C2F3834223
:103F8000113202E0022404EB924213B14B689B030E
:103F900001D5064B00E0024B5A43C0E70010024037
:103FA00000127A000400002000003C0800093D00D7
:103FB0002DE9F041274CA61540212046FEF794F943
:103FC000850080212046FEF78FF945EA40053146FD
:103FD0002046FEF789F90543EDB240212046FEF761
:103FE00083F9870080212046FEF77EF947EA4007E3
:103FF00031462046FEF778F90743F8B2A842DBD1F4
:1040000040212046FEF770F9870080212046FEF708
:104010006BF947EA400731462046FEF765F907434A
:10402000F8B2A842C8D140212046FEF75DF98700CA
:1040300080212046FEF758F947EA400731462046DE
:10404000FEF752F90743F8B2A842B5D12846BDE8B9
:10405000F08100000010014010B50268416802FBC9
:1040600002F301FB01330D4CA34211D91B0E0E3B91
:104070000B4C9BB212B234F8133009B25A43594375
:1040800042F38F3241F38F31C0E90221012102E076
:10409000C0E902210021017410BD0000E10BBF0E38
:1040A000B88700082DE9F05FFE48FF4902880B88B9
:1040B0009A1A92B20F2A79D309880180FB480246E6
:1040C0008189D2884B0703D48B0701D4CB0702D058
:1040D00042F4007201E022F40072C28081460807B7
:1040E00002D44846C90604D5B9F8061041F00101CA
:1040F00002E0C18821F00101A9F80610EB48FDF7A4
:104100009DFEEB494FF4804AB1F93A00504502DA7E
:10411000401C488701E0A1F83AA0E64E41F6CC41A8
:10412000E54DB06C884203DDA86820F01000A8605F
:10413000E249E34FDFF88CE30888002410B1401E09
:10414000088008E0E88F40B1401EE887DE4801782B
:1041500021F002010170EC7330E0B9F8060042046E
:104160001BD4B9F80C10CA0617D4090715D40106D8
:1041700013D4810611D401050FD4410603D5D349C8
:104180000978090609D5410707D4C10505D40107F7
:1041900003D4810401D4C00609D5CD48EC73CD49C0
:1041A0003C70C4830C8080F82A4008E087E03878AF
:1041B000012804D19EF80000062800D13C70387810
:1041C000DFF8F4B24FF00108ABF12C0B0A2878D2DB
:1041D000DFE800F0F5750575F4F37577DFFAE87B35
:1041E00009281AD0DFF8F092022875D0B5F84000FF
:1041F00010B399F8680040F63A22012822D0C5F899
:10420000D84085F8EA40CBF82040B5F9301001F2EB
:104210001D50904226D8102325E0A2484430FEF7D6
:104220004FF9FDF785FE716CCBF8281041F27C51F7
:104230000920CBF818109FE1A84841892986A5F8E4
:10424000408015E0A648C5F8D80085F8EA80B5F9A1
:10425000301001F21D53934201D8102300E02023B7
:10426000102202E020231022002000F029FB2886E3
:1042700099F868309B49012B736C40F2DC504FF485
:10428000927211D0834204DA9448B0F90A00904245
:1042900011DBB5F8402040F6C410521C92B2A5F8CC
:1042A0004020824207D20EE0834208DA8B48B0F900
:1042B0000A00904203DA3C7085F8EA404C83BDE87E
:1042C000F09FC8E008E0854800890028F7D18648BB
:1042D00000780128EFD0F2E7706CCBF828008BF85B
:1042E0000780824FA5F8404085F8EA40797F5E4616
:1042F00099B1F87FE0B3288DB5F9301000B20A23E8
:10430000052200F0DDFA2886FC777C77B5F93000CD
:1043100050453ADDA5F830A0D1E700B2744901F06C
:1043200025FCA5F8E400A96A814200DA084600B23B
:10433000B08299F84D100029B5F9301002D036231B
:10434000052202E040F24713102200F0B9FA288655
:10435000B5F91601B5F9141188420ADA317901F17B
:104360000101C9B231710429D0D33471401C02E07B
:1043700007E003DD801EA5F81601C7E7A5F81611B2
:10438000C4E740F266602886C0E7002897DA2C86EA
:1043900095E75848D5F8DC10814202D2491CC5F88F
:1043A000DC10E97B082903D1D5F8DC10814207D362
:1043B0003C70C5F8DC4082E706E02BE026E02EE00A
:1043C000BDE8F05F02F02EBCE87B092801D02C8606
:1043D00045E1DBF81C005F46401CCBF81C000228BE
:1043E00009DD388D012301B2388B052200B200F0BF
:1043F00067FAFC61B8622B48398D44300180B6F809
:1044000044104180FEF774F8288658E7BDE8F05F55
:1044100004F094B838480078092877D04FE7374936
:10442000374B0888401C82B236480A80C82A04D319
:1044300090F800C0BCF1010F19D0B2F57A7F04D317
:1044400090F800C0BCF1020F11D0B2F5FA6F02D3A0
:104450000278032A0BD0E87B801E08287ED2DFE892
:1044600000F011C3FDFC057D9C04D6E627E704702F
:104470000C80B9F8061021F40061A9F8061083F841
:104480000080E8E7FDF76AFF3078400647D51E4810
:104490008078042843D0706C822840DAB07A00F02B
:1044A000030034E01C090020FC0600200C0A002058
:1044B00020050020400100209C0200200007002071
:1044C000F3060020F4060020CA050020D4060020D0
:1044D000B00800201E000020600C002060000020BA
:1044E0009AF9FFFF8C09002038010020280C0020D9
:1044F0004A890008C0D4010058020020160000209C
:10450000140000201500002040040020A7E096F8C9
:104510003D1001F00301884201D001F027FD3878F9
:104520000628A3D086F83F40B06C614940F31100E3
:10453000C86281035F480162FDF7FAFC8BF80780CF
:10454000B5F81401A5F81601706CA5F88240B0F515
:10455000437FA5F880A011DDA86800E09FE040F44B
:104560008060A86096F8381005297FF4B4AE00BFCB
:1045700040F01000A8606EE03870A0E6A96821F451
:104580008061A96040F28A21884204DA30784006CE
:1045900001D402F033FAA868EAE7706CB0F5437F03
:1045A00007DA9EF80010062903D000BF8EF80040FD
:1045B0006DE04148017821F040010170FDF7B8FC41
:1045C000A5F816A1FDF7CAFE3C4810F8281F21F0F7
:1045D000010101703A49C5F8DC400C6235490C62B2
:1045E0000821397044646AE699F80600C006C4D40C
:1045F000706CB0F57A7F32DDFDF7B0FE30784006A2
:1046000011D53048807804280DD0706C82280ADAE1
:10461000B07A96F83D1000F0030001F003018842E3
:1046200001D001F0A3FC86F83F40B6F84800288688
:1046300001B22C46514501DDA4F830A0FDF778FC0D
:10464000A06840F48060A06096F83810052994D1E5
:1046500040F01000A06002208EE714E001E03C7002
:104660002DE6706CB0F5437F03DA9EF80010062942
:104670009CD1B9F8061021F02001A9F80610FDF729
:104680006DFE042078E79EF80000062802D087F827
:10469000008014E60C490920087005206CE70948E1
:1046A000847003488EF8004080F856406FE60000A2
:1046B000600000208C08002002070020200A002053
:1046C00068080020400400205802002030B585B062
:1046D00001210420FFF700FC4FF40040ADF810006A
:1046E00048208DF8130004A91848FDF77FFD01212B
:1046F0000846FFF7D9FB40F68C20ADF804000324F0
:104700000020ADF80040ADF80200ADF806004FF013
:1047100080456946284600F0B9FF1C208DF80C0042
:104720008DF80D408DF80E4001208DF80F0003A884
:10473000FFF792F801221146284600F081FE012180
:10474000284600F0AFFD05B030BD00000008014074
:10475000704700002DE9F041304CE07800285AD134
:104760002078002857D0401E10F0FF00207052D152
:104770004FF49670208272B6294F45F2AA50A7F8DE
:1047800072000020FDF7B2FB264D13202860FDF7D4
:10479000BFFBA8BB3420E86002202861224E6E6176
:1047A000286940F040002861FDF7B2FB40BB0021C2
:1047B0001E4A08465FEA255312F800C0BCF1FF0FFD
:1047C00000D00121401C80B29842F5D3C1B9C4E9A0
:1047D000067639260127A06910F8011B10F8012B75
:1047E000A061E06901EB022102886A612F6120F873
:1047F000021BE061FDF78CFB10B9761EB6B2EAD25F
:104800000120FDF773FB62B601F004FC08488168E3
:1048100021F480418160BDE8F0810000F0060020B5
:10482000600C00200020024000FC000800FC000892
:104830009C0200201948016841F0100101600168E4
:1048400021F003010160016841F002010160144898
:104850004168416041684160416841F48061416064
:10486000416821F47C11416041680E4A1143416066
:10487000016841F08071016001688901FCD54168DF
:1048800021F003014160416841F00201416041684B
:10489000C1F381010229FAD17047000000200240D3
:1048A000001002400000280830B5044C039D6080D1
:1048B000A180E2802381658130BD0000000A0020D4
:1048C0000A44824201DA10B27047C91A8142FBDD04
:1048D00008B27047F0B53E48DFF8F8E03E4CC17FC3
:1048E000467A056800233D4A3D484FF0010C802977
:1048F00025D301F01F015EF821100D420146096821
:1049000002D041F4805101E021F480510160CF04D4
:1049100011D48F040FD5977AFF0705D053812778DC
:1049200027F00207277006E090F846709FB1012F2C
:1049300014D080F846300F0B67F34D310160802EA4
:1049400025D306F01F015EF821100D42016809D041
:1049500041F0040108E080F846C0ECE7022780F847
:104960004670E8E721F0040101604D070BD44D05C6
:1049700009D5957AED0706D05381257825F00205F3
:104980002570C0F898308C0864F38A210160917A10
:10499000C90718D1134991F86410012913D112499C
:1049A000496C32290DDC017849070AD501890905CE
:1049B00007D4D0F8981047F23054A14204D9A2F895
:1049C0000AC0C0F89830F0BD491CC0F89810F0BD7E
:1049D000D0050020708E0008CA0500200C0A0020B7
:1049E0009C020020600C00204001002010B5FCF764
:1049F000C1F90F48018821F0020101800C491831EA
:104A000009880C4A928E1144094A343211800849AF
:104A10000C390A8842F001020A80011D0A884FF60B
:104A2000ED531A400A80018841F01201018010BD47
:104A30000C0400404004002006480188491C89B24B
:104A40000180B1F57A7F04D34188491C418000215F
:104A500001807047140700200F4810B5016841F02D
:104A60000101016041680D4A1140416001680C4A32
:104A700011400160016821F480210160416821F446
:104A8000FE0141604FF41F018160FFF7D3FE05492D
:104A90004FF00060086010BD001002400000FFF8F9
:104AA000FFFFF6FE08ED00E02DE9F0412F4D2888CC
:104AB0004FF00004000629D5FCF7D8FA2C4A2D48FF
:104AC00007231778C8262C49012F22D02B4FB7F87F
:104AD00006C0BCF1000F3ED0B0F80CC04CF0080C82
:104AE000A0F80CC0B0F806C02CF4006CA0F806C00A
:104AF000886820F004008860FC801370CE87002056
:104B00004FF49661401C80B28842FBD32C80BDE8F4
:104B1000F0811B4F97F800C0BCF1010F0FD0BCF122
:104B2000020F11D0B0F806C04CF4006CA0F806C01B
:104B3000886840F00400886005203870DDE7B0F830
:104B40000CC04CF0080C03E0B0F80CC04CF0100C9A
:104B5000A0F80CC0F0E70B4F3C70C78847F4006723
:104B6000C780886840F004008860C6E7102C0140C8
:104B7000F30600200C0A00209C0200201C090020E3
:104B8000F406002011070020704700002DE9F043D3
:104B90004FF08040018A21F001010182AC48007889
:104BA00000287CD1AB4FF87B002878D1AA48406C14
:104BB000322874DCA9488068DFF8A4924104A94D2A
:104BC000B9F804004FF0000403D4401CA9F8040015
:104BD00028E1002874D02978012611B1012912D0CA
:104BE00017E14946B0F5BE7FFAD92E70CC718C71B1
:104BF000EC702C72287A0A18401CC0B21472287209
:104C00000F28F7D305E1B9F802204946824201D9BD
:104C1000EE7100E0EC7192488A7908300F2A15D2C3
:104C2000CB79082B0BD2C3F10708EB7912F800C03F
:104C300003FA08F363441354CA79521CCA71CA793F
:104C4000082A03D18A79521C8A71CC7199F806100E
:104C5000C8460F2973D10D21FCF772F9A881010A0A
:104C60006970C0B2A87088F8064098F816208A4289
:104C700065D198F81510814261D198F80BC07A4936
:104C8000032302227948BCF1000F10D0BCF1010FC0
:104C900002D0BCF1020F14D080F86A2000E0CBE013
:104CA00091F800C02CF00C0C0CF1080C0FE080F80F
:104CB0006A6091F800C02CF00C0C0CF1040C06E0BA
:104CC000A9E080F86A3091F800C04CF00C0C81F833
:104CD00000C098F80C10B6EB111F04D180F86E409C
:104CE00087F846400EE0B2EB111F04D180F86E60E9
:104CF00087F8466006E0B3EB111F03D180F86E2001
:104D000087F846200B0717D001F00F01012901D0C9
:104D1000022915D080F86C602C7198F80D102A7952
:104D200006FA02F30B406B71082A44D2DFE802F066
:104D30000B124319242F363D80F86C40ECE768E0F5
:104D400080F86C20E8E713B180F8704033E080F819
:104D5000706030E013B180F850602CE080F8504073
:104D600029E023B180F8656087F8036123E080F8CB
:104D7000654087F803411EE023B187F8F54080F8CD
:104D80004D4018E087F8F56080F84D6013E013B1EE
:104D900080F868600FE080F868400CE013B180F89C
:104DA000666008E080F8664005E013B180F867604F
:104DB00001E080F86740521CD2B22A71082AAED3B3
:104DC00098F80E102A4A8B0705D587F8F16080F80D
:104DD0006460568104E087F8F14080F864405481B3
:104DE000C90702D080F8294001E080F8296098F8CE
:104DF000111000F86D1FC2781E48012A1ED001B3A1
:104E0000012921D04FF48051A0F876101A493C2096
:104E10000870A9F80240A9F80440B9F80210491C2A
:104E2000A9F80210B9F80210B1F5FA7F04D940F2DE
:104E3000F511A9F802102C70BDE8F08344F21C7142
:104E4000E2E74FF40051DFE741F25551DCE70000A3
:104E5000F30600209C0200204001002000100140C9
:104E6000480C00208C060020B8040020600C0020B4
:104E70000C0A002020050020F00600202DE9F05F3C
:104E8000FDF76CFA8E4D2888A5F10406C0070AD0FC
:104E9000308820F008003080288820F00900288021
:104EA00001F0ACFDD9E02888DFF81892DFF818820D
:104EB000864C80071AD5B9F8001041F00101A9F815
:104EC0000010B8F80000804914315030088028885C
:104ED0004FF6F95108402880308840F004003080B7
:104EE000FFF766F884F83C00BDE8F09F2888784F0B
:104EF0004007288871D520F004002880FFF758F873
:104F000094F83C108142EFD1308820F004003080CA
:104F1000FDF7FCFB2078410605D594F84C1094F879
:104F20003B209142E0D03978400621F002013970EF
:104F300004D5FEF7F5FA97F82F7004E094F83C00DA
:104F4000FDF75EFA0746DFF880B140F68C2A0BF1D8
:104F5000180B062F47D294F83800B8423ED0384696
:104F6000FDF7D2F92078C00716D094F83A0094F8EB
:104F7000391000F00302914206D0A17A00F001003E
:104F800001F00101884215D1FDF728FBFBF73EFF38
:104F9000FDF750FC384689E0FDF720FBFBF736FFB4
:104FA000FDF748FC3846FDF739FB207840F001005A
:104FB000207099E7288820F008002880206B81085D
:104FC00001EBD000504515D2B8F800100844ABF8FA
:104FD0000000308840F0080003E00DE0308820F049
:104FE0000800308080E7B9F8001041F00101A9F80D
:104FF0000010DFE75046E7E70007288831D520F0AA
:1050000008002880308820F008003080FEF7D0FFAC
:1050100084F83C00FDF77AFB387820F00200387005
:105020002078400604D5FEF77BFA97F82F5004E06D
:1050300094F83C00FDF7E4F90546062D08D294F8F3
:105040003800A842B5D0FDF7C9FAFBF7DFFE2AE029
:105050002048C18841F04001C180BDE8F05FFDF704
:10506000C9BBC006288825D520F0100028803088CC
:1050700020F01000308097F838000C2802D2401C35
:1050800087F83800387840F002003870FEF748FAA8
:1050900097F82F50787884F8390094F83800A842AF
:1050A00087D0FDF79BFAFDF7C5FB2846BDE8F05F0A
:1050B000FDF7B4BA4EF2BE110840288014E7000094
:1050C000100400400004004024040040400100207F
:1050D000400400200C0A00202DE9F04F514F85B00C
:1050E000388820F0010038804E48002610300680B5
:1050F0004D4CDFF838A14FF0010894F85C0042F6FF
:105100003029C10774D072B64948816941F40071F1
:105110008161816941F4806181614FF40040FEF753
:10512000ADFE444D00212846FBF7CEFB002128466A
:10513000FBF7C0FBDFF800B100215846FBF7BAFBD4
:1051400000213E48FCF752FA2846FBF7D9FC5846A6
:10515000FBF7D6FC4FF46020CDE902068DF8056020
:1051600000968DF810808DF8048069462846FBF77C
:1051700059FD01231A460F212846FBF7A4FD012102
:105180002846FBF797FB00204946401C80B2884226
:10519000FBD328462E600121FBF7D4FD2868800749
:1051A000FCD524484C30006894F85C1021F00101D3
:1051B0002144A1F85000FBF791FB62B6FEF7BCF862
:1051C00047F69061AAF8001094F85C00401CC0B249
:1051D00084F85C000C2822D212491431A1F8008016
:1051E000388840F00100388005B0BDE8F08FFFE757
:1051F000134920F00100085A12490880114945F668
:105200005800083908800F4847F25801001F0180F4
:105210000C4920200C390880AAF80090D4E703201C
:10522000A070E1E700080040400400202C08004086
:105230000010024000240140002801400800024004
:105240002C8A0008202C01400029018802D041F05E
:10525000800101E021F080010180704710B50A88CB
:105260004B88CC881A438B8823431A430B891A43F3
:105270004B8989891A430A43A0F8442010BD0021B4
:10528000018041808180C18001814181818170479D
:105290000029818802D041F0010101E021F00101E3
:1052A000818070470029018802D041F0010101E0AE
:1052B00021F0010101807047002930F8441F02D01D
:1052C00041F4004101E0C1F30E010180704700008C
:1052D0004B4910B5884202D10121C41486E0B0F1D7
:1052E000804F09D0474988420DD101210220FEF7A5
:1052F000E7FD0021022064E001210846FEF7E0FD01
:10530000002101205DE04049884206D101210420AE
:10531000FEF7D6FD0021042053E03C49884206D127
:1053200001210820FEF7CCFD0021082049E0384982
:10533000884206D101211020FEF7C2FD0021102075
:105340003FE03449884206D101212020FEF7B8FD14
:105350000021202035E03049884202D10121441447
:1053600044E02E49884202D10121CC043EE02C4980
:10537000884202D101210C0538E02A49884202D135
:1053800001214C0532E02849884206D10121402004
:10539000FEF796FD0021402013E02449884206D103
:1053A00001218020FEF78CFD0021802009E02049AA
:1053B00088420AD1841501212046FEF781FD002193
:1053C0002046BDE81040FEF77BBD1A49884202D155
:1053D00001210C040AE01849884202D101214C0441
:1053E00004E0164988420AD101218C042046FEF7C8
:1053F0007FFD2046BDE810400021FEF779BD10BDBD
:10540000002C01400004004000080040000C004057
:10541000001000400014004000340140004C0140E6
:10542000005001400054014000180040001C0040A2
:10543000002000400040014000440140004801407D
:10544000002A828901D00A4300E08A4382817047A2
:1054500030B5028C22F001020284028C8388048B16
:1054600022F0020224F073050C882C430D891543A9
:105470004A882A43114DA8420BD0114DA84208D0AA
:10548000104DA84205D0104DA84202D00F4DA842A1
:105490000DD122F008054A8923F440732A4322F0F3
:1054A00004058A882A438D891D43CB892B43838039
:1054B0000483C9888186028430BD0000002C01402D
:1054C00000340140004001400044014000480140D8
:1054D000028B22F008020A430283704770B5028CE7
:1054E00022F010020284028C8488038B0D8823F43E
:1054F000E6464FF6FF7303EA052535430E8922F091
:10550000200203EA061616434A8803EA02123243CF
:10551000104EB04202D0104EB04215D122F080069B
:105520004A8924F4406403EA0212324322F040061E
:105530008A8803EA021232438E8903EA86062643EA
:10554000CC8903EA8404344384800583C9880187B5
:10555000028470BD002C014000340140028B4FF6E4
:10556000FF7322F4006203EA0121114301837047B3
:1055700070B5028C22F480720284028C8488838B42
:105580000D8823F073031D4322F400730E894FF638
:10559000FF7202EA06261E434B8802EA03233343C6
:1055A000104EB04202D0104EB04215D123F4006626
:1055B0004B8924F4405402EA0323334323F48066E6
:1055C0008B8802EA032333438E8902EA06162643B8
:1055D000CC8902EA0414344384808583C988818796
:1055E000038470BD002C014000340140828B22F006
:1055F00008020A438283704770B5028C22F48052FD
:105600000284048C8288838B0D8823F4E6464FF64F
:10561000FF7303EA0525354324F400560C8903EA99
:10562000043434434E8803EA06362643094CA0422C
:1056300002D0094CA04205D122F480448A8903EAB1
:105640008212224382808583C988A0F84010068494
:1056500070BD0000002C014000340140828B4FF6E9
:10566000FF7322F4006203EA012111438183704732
:10567000018582827047828822F07002828082884F
:105680000A4382807047A0F84010704730B5028806
:105690001B4B1C4C98420DD0A0420BD0B0F1804F58
:1056A00008D0194DA84205D0184DA84202D0184D77
:1056B000A84203D122F070054A882A43154DA8421A
:1056C00006D0154DA84203D022F44075CA882A435B
:1056D00002808A8882850A88028598420AD0A04280
:1056E00008D00E4A904205D00D4A904202D00D4A91
:1056F000904201D1097A01860121818230BD0000EA
:10570000002C01400034014000040040000800402B
:10571000000C004000100040001400400040014018
:1057200000440140004801404FF6FF718180002194
:105730000180C1804180017270470029018802D038
:1057400041F0020101E021F00201018070470029CF
:10575000018802D041F0040101E021F00401018040
:1057600070470000204810B590F82010026801F042
:105770001F001E4951F820001D490242086802D04E
:1057800040F4803001E020F48030086019484FF088
:10579000000280794106184824D4184903880C88EF
:1057A000E31A9CB201230F2C08D30C880480846870
:1057B000042C03DD124C2478022C05D0427F012AF0
:1057C00006D00988418010BD4377C2770A8842809D
:1057D00042880988891A89B240F21A629142F2D34A
:1057E000C37710BD427710BDD0050020708E000831
:1057F0009C0200200C0A0020280C0020FC0600203F
:10580000F30600202DE9F04FDFF8B8B16A48DFF861
:10581000AC91DFF8ACA190F80EC0BBF91A70BBF9DF
:105820001C60BBF91850BBF96C10BCF1070F48D2D3
:10583000DFE80CF08D041A30485E7600D9F80020BD
:105840008284DAF80020C284828CC38CA7EB8202A7
:1058500012B2A6EB83034A431BB2594342F3CF2251
:1058600041F3CF23D11870E0D9F800204284DAF850
:105870000020C284428CA5EB820213B2C28C4B433F
:10588000A6EB820212B243F3CF24514341F3CF235C
:10589000E11814E0D9F80020C284DAF8002042842C
:1058A000C28C438CA6EB820212B2A5EB83031CB21E
:1058B0004A43614342F3CF2341F3CF2419194942AC
:1058C0000AB244E0D9F800208284DAF80020428449
:1058D000828C438CA7EB820212B2A5EB83034A436E
:1058E0001BB2594342F3CF2241F3CF24111914E0E4
:1058F000D9F800204284DAF800208284428C838C1C
:10590000A5EB820212B2A7EB83034A431BB242F318
:10591000CF24594341F3CF22A11849420BB216E0DC
:10592000D9F80020C284DAF800208284C28C838CEB
:10593000A6EB820212B2A7EB83031CB24A4342F3E6
:10594000CF23614341F3CF22991849420CB2BBF9EE
:105950001E50594605F21E56A64201DACE8306E0D5
:10596000A5F21E55A54201DDCD8300E0CC83B1F93F
:10597000204004F21E55954201DA0D8406E0A4F29F
:105980001E54944201DD0C8400E00A84B1F9222007
:1059900002F21E549C4202DAABF8224008E0A2F266
:1059A0001E529A4202DDABF8222001E0ABF8223011
:1059B000417B8173BDE8F08F9C0200203C240140B4
:1059C0003C280140200500202DE9F04704465C48B2
:1059D0005D4D002602785B48022AB0F9301004D0F1
:1059E000082A70D0092A6FD0A5E0C27B022A02D112
:1059F000B0F840204AB1E18769810423B5F9081065
:105A00001A460020FEF75CFF8CE05049DFF8408129
:105A1000496A0F14E7808068410210D5B4F902008A
:105A200040F2DA21884269DD40F26A4188423FDC77
:105A3000A0F2DA20FAF7F3FC0022464B4DE0C0F367
:105A4000C001C0F30020DFF8109181420CD1D8F8DA
:105A5000440040F2BA41884250DD40F66A11884263
:105A600026DCA0F2BA4034E03C480078C0060CD5F1
:105A7000D8F8440041F2243188423FDD41F2D4712C
:105A8000884215DC00F6DC4021E0354890F87010C3
:105A9000012903D090F86F0001282FD1B4F902003A
:105AA00041F6C811884229DD41F6786188420CDD53
:105AB0000823B4F93E101A460020FEF701FFE087E4
:105AC000002819DB1BE02FE033E000F5C760A0F5EC
:105AD0000050FAF7A4FC00224B46FAF70CFC0E2209
:105AE000FAF778FCFAF7D2FC00B2C0F580407843B0
:105AF0008013E087002F02DCE68700E0E787E08F75
:105B0000184FE880D8F844107964A7F84C0000F0EA
:105B10007DFBB7F84E00688198F80A000028388F9E
:105B200000D14042288106E00F48B0F8700068813B
:105B300000E069812E8184F83C60BDE8F0870000B8
:105B4000F30600209C0200206000002020050020B9
:105B5000400100200000794000C09240D40600209F
:105B6000600C0020B0080020200A00202DE9F04140
:105B7000B1F9025000232B241522854203DAB1F932
:105B80000000BDE8F081B1F9AE50854202DDB1F907
:105B9000AC00F6E701EB8205B5F90250854201DD64
:105BA000134600E01446E21852085D1CAA42F1D1E7
:105BB00001EB8206B6F90230834206DA36F9025C5E
:105BC00036F9044C31F9221006E01D4631F9224025
:105BD000B6F90630B6F90410401B091BC617891127
:105BE000B60346EA90468703A1FB070CCA1702FBDF
:105BF00007C201FB06215A1BD317FAF795FA000AD0
:105C000040EA0160001900B2B0F5804FB9DB43F6FD
:105C1000FF70B6E770B5134C40F224452946204684
:105C200000F03EF800281BD0204600F0C7F82946B7
:105C3000204600F01DF80C4C00212046FBF7D6FC56
:105C40002046FBF751FDC0F164000849C0B20428AA
:105C5000087201D900F046F9BDE87040FBF78ABD33
:105C600070BD000000380140580002405C06002072
:105C70000A0A01219140C9430180704700298189A6
:105C800002D041F4005101E021F4005181817047BC
:105C9000002A828A01D00A4300E08A438282704748
:105CA00030B501F01F0201240025C1F3421304FAAC
:105CB00002F2012B0FD0022B0FD0838A4FEA112161
:105CC0000088134204FA01F400EA040001D000B194
:105CD0000125284630BD8389F0E7038AEEE710B539
:105CE000C1F3421301F01F040121A140012B07D091
:105CF000022B07D01430002A026805D00A4304E0C2
:105D00000C30F8E71030F6E78A43026010BD00005F
:105D100030B50446008A85B00D464CF6FF71084048
:105D2000E98801432182A1894EF6F3100140A88839
:105D30002A8910436A890A431043A081A08A4FF63A
:105D4000FF410840A9890143A1826846FEF7DCF8BB
:105D50001948844201D1039800E00298A1890904FE
:105D600000EBC00101EB0010296801D5490000E0FB
:105D70008900B0FBF1F06422B0FBF2F109010B09DC
:105D80006FF018056B4300EB8300A3891D044FF0EF
:105D9000320306D503EBC000B0FBF2F000F00700C1
:105DA00005E003EB0010B0FBF2F000F00F00084339
:105DB000208105B030BD0000003801408088C0F36C
:105DC00008007047F8B501210920FEF785F8012188
:105DD0008803FEF781F810258DF803502020ADF8D8
:105DE00000001A4E03248DF8024069463046FCF745
:105DF000FDF916490C31086820F0200008601820D1
:105E00008DF803004020ADF800008DF8024069468F
:105E10003046FCF7EBF948208DF803008020ADF800
:105E2000000069463046FCF7E1F98DF8035028017F
:105E3000ADF800008DF8024069463046FCF7D6F90F
:105E400001210420FCF724FAF8BD0000000C0140F9
:105E500030B585B0FFF7B6FF00244FF4E130009075
:105E6000ADF808400C201D4DADF80440ADF80A0017
:105E7000ADF80640ADF80C4069462846FFF748FFEC
:105E800025208DF8100004208DF811008DF81240A7
:105E900001208DF8130004A8FDF7DEFC012240F27A
:105EA00024412846FFF71BFF01212846FFF7E6FEA5
:105EB000FBF78AFC012280212846FFF7E9FE012238
:105EC00040212846FFF7E4FE012202210448FBF7A7
:105ED0001FFCFBF779FC05B030BD00000038014025
:105EE0004400024070B51D4D00242878432834D169
:105EF0006878462831D1A878502807D0512805D095
:105F0000812803D0892801D0212826D1144E707110
:105F1000E9787172A81C891CFBF74AF8B072717A93
:105F2000294409793182884217D106F10E0001789F
:105F300041F0020101700B48016841F0200101604D
:105F4000317A0948002204E02B5D03552A55641C70
:105F5000E4B28C42F8D38078707170BD880700205D
:105F60005C0600200C0C0140920B002070B51D2037
:105F7000FDF751FCFDF7D4FA1D20FDF762FC154832
:105F800090F82F10144D0623144C85F8381090F813
:105F90003B1095F83B201143012A04D0022A07D078
:105FA000042A0AD010E0827A8A420DD0007B09E0F0
:105FB000027D8A4208D0807D04E0827F8A4203D03D
:105FC00090F82000884200D12370002085F840001E
:105FD00070BD00004004002040010020F3060020B6
:105FE0000B4800214180A0F1B0018A898280CB89D1
:105FF0001A44C2800B8A1A4402814B8A1A44428195
:10600000898A1144818143F6FF71C1817047000084
:10601000F0010020084940F61C72B1F90C009042D2
:1060200002DA00F59F7005E041F2E302904201DDE3
:10603000A0F59F70C88170476000002038B51348F4
:10604000C16941F00401C1611E208DF800000220E9
:106050008DF801008DF8020001248DF80340684698
:10606000FDF7FAFB0A4984200880094947F6906049
:106070002C3108800020091F0880054914310C804C
:10608000091F0880081F048038BD0000001002406E
:106090000008004030B420491E4A45788B7A1146EA
:1060A00092F83B4091F83910AC4218D14BB10379CA
:1060B000994202D04379994201D140791AE080791E
:1060C00009E08379994202D0C479A14202D182F8D1
:1060D0002F3011E0407982F82F0030BC7047C5782E
:1060E000AC42FAD16BB1C379994202D0037A99429A
:1060F00005D1007A82F82F0030BCFEF777BC407AD9
:10610000E9E7437A9942E2D00479A142DFD0007AEC
:10611000E1E700004004002040010020FEE700000D
:106120002DE9F0470446007F012868D13548E18811
:106130000288511A89B2072916D30088E080B4F981
:10614000000044F2DD414843401346F6D96148431C
:106150008013A060401000B2A0814FF08051B1FBCD
:10616000F0F0FAF757F92061B4F90C6096B1B4F980
:1061700002104DF6B05048430014A082B4F90470E8
:106180004DF6B05207FB02F24FEA2245E58204D4F5
:10619000024603E00020E08330E0424212B2228354
:1061A000002D01DB2B4600E06B421BB2DFF858905C
:1061B000638398464FF4804AB24208DAFAF721F92D
:1061C0002169F9F7F4FFFAF748F9801304E0002990
:1061D00001DA484600E05046E083B04509DA284637
:1061E000FAF70FF92169F9F7E2FFFAF736F98013A8
:1061F00004E0002F01DA484600E050462084BDE864
:10620000F0870000FC06002000C0FFFF70B52E489C
:1062100000252F4C01782D48022905D1C17B022988
:1062200002D1B0F8401021B1008EA4F84E002587AD
:1062300070BD90F8462026482649022AB0F844004E
:10624000097800B2C1F3810103D0012A0DD022499F
:1062500014E0012904D0022904D01F4960390DE05F
:106260001E490BE01D49603108E0012904D00229D4
:1062700025D01949303901E018493031FBF706FEC5
:106280001349A4F8400080B2483101F085FAB4F90E
:106290004C00B4F94A204142514341F38F3124F874
:1062A000381F01F5FA71B4F9102050438013E082D1
:1062B0000B48B1F57A7F05D90121017070BD0649FF
:1062C0009039DBE7057070BDF30600209C020020CA
:1062D000B0080020B8040020FC880008DC87000813
:1062E000380100200348002180F82A10C18301876B
:1062F00070470000B008002010B504000B462D4A7E
:10630000C3F1000028D56442002B12DAA04207DA5C
:10631000214600F027FA32F81000C0F5404041E075
:106320000146204600F01EFA32F8100000F5004049
:1063300038E0A34208DA2146184600F013FA32F892
:10634000100000F540402DE0204600F00BFA32F836
:106350001000C0F5803025E0002B12DAA04207DAE9
:10636000214600F0FFF932F8100000F5804019E0F6
:106370000146204600F0F6F932F81000C0F5004062
:1063800010E0A34208DA2146184600F0EBF932F893
:106390001000C0F5804005E053B1204600F0E2F95E
:1063A00032F81000B0F5004F01DDA0F5803010BDCF
:1063B000002010BD388A000840438013494300EB99
:1063C000A13000220302002B14DDB3F5001F01DC15
:1063D000802001E04FF4005093FBF0F1014401EB09
:1063E000D1714910814206D0521CD2B20846062A09
:1063F000F2D300E00021C80000B2704702E008C8F4
:10640000121F08C1002AFAD170477047002001E02E
:1064100001C1121F002AFBD1704700002DE9F0478F
:10642000A44CA54821880288511A89B20F297DD32E
:106430000088A4F13C052080288F08B1401E2887E1
:106440002B789E4AC3F3810001281DD0022820D05A
:10645000D18B98489A4FDFF86C92407E0026B1F5B8
:10646000926F1DD8142819D378206076F88840F0F0
:106470001000F88040F26660A88123F001002870C7
:10648000D67389F8006015E0D08B00EB4000C003A4
:1064900002E0D08B8C494843010CDAE7401C04E051
:1064A000B1F5DB6F06D310B1401E607602E043F019
:1064B00001002870B5F90200B5F914304143C3EB6F
:1064C000C303C1F38F31C3F3D10303EB510109B20D
:1064D000A9829046D28B4FF080535043B5F91620D5
:1064E000C0F38F30C2EBC202C2F3D10202EB500004
:1064F00000B2E882AA6A42431213EA6293FBF2F204
:106500002A63724A1080A2680A44A260E1680144CA
:10651000E160207C401CC0B22074072806D942F3F9
:10652000CF002883C9106983E66000E0BFE0A66061
:1065300041F6C8012674884204DD298B644AB2FB07
:10654000F1F1E981C117890341EA9041800342F6E4
:106550009B420023F9F7E8FDA88456482A78A0F169
:106560003C005C49B0F90600930700FB01F14FEADB
:106570002141C2F3810215D5012A07D0022A0BD08E
:106580004FF2685141430914A18011E049F68C4251
:1065900050430014A0801FE04CF618314143091409
:1065A000A18025E0012A0DD0022A17D0A08069849D
:1065B000494948430014E083FBF788FA47480088BC
:1065C000C0B143E04AF65C3242431214A2804BF65B
:1065D0002C22504300146884E183EDE74DF2AC5166
:1065E00041430914A1804EF27C414143091469845E
:1065F0003B49DEE795F8200000BB88F80F6089F87A
:106600000060B5F91A00A0F50C519F39B1F56E7F05
:1066100018D8617FF42912D93249E8802E4AA1F8AE
:10662000460050430014A880A1F84400FF2085F8DC
:10663000200081F828002C493C20087006E0491C05
:10664000617703E0607F08B1401E6077B5F91A10EA
:10665000B4F91E0081420EDDA07E7D2809D9F8889C
:1066600040F00800F8802148017821F00201017013
:106670000EE0401C06E0A0F23D10814208DAA07E48
:1066800010B1401EA07603E0F88820F00800F880E2
:10669000B5F91810606908446061217E491CC9B2CF
:1066A00021761F2903D94011A88366612676BDE8AB
:1066B000F0870000F4040020FC0600209C0200206B
:1066C0000C0A0020F306002030330100C00900202E
:1066D00074E8260BCC0E010048850100FE06002060
:1066E000D0450100600C0020F0060020CA05002003
:1066F000024941F68B30886270470000B8040020E0
:1067000070B5164C06252078062825D2DFE800F063
:1067100003080E141A211248FAF788FC012016E02B
:106720000F48801DFAF782FC022010E00C480C3064
:10673000FAF77CFC03200AE009481230FAF776FCED
:10674000042004E006481830FAF770FC0520207099
:1067500070BDFAF78BFC2570257070BDF406002023
:106760002C890008090A05D0B0FBF1F0FF2800D9F8
:10677000FF20704700207047D0E90021C368521AFB
:106780005A4301EBA231816041607047B0F90020AB
:10679000B0F90210B0F90630521A5A4301EBA23197
:1067A000818041807047000030B5444B18884449CF
:1067B0008A89801A85B24348434A0F2D047801F133
:1067C0004C001DD31D888D81117A090713D5022C29
:1067D00001D03E4912E03E4DB0F90210B5F900502B
:1067E000A94205DC02DA01F1020108E0458007E078
:1067F000A1F1020103E0022C02D13649098841804F
:10680000018F1D88691A89B29C2942D31988018792
:10681000916A0023B1F5804F2DDB2F49896CB1F5CA
:10682000405F28DD2D4940F26665B1F91010A9429C
:1068300011DD43F69915A94202DB40F2333108E03D
:1068400040F23335A1F26661694343F2333591FB7F
:10685000F5F1818700E083872149B2F80651097874
:10686000C1F381011DB1818F01F21E5119E092F82F
:106870004620022A0ED08387022C00D08387B0F9ED
:106880005410B0F93C3001F114029A420BDAA0F82E
:10689000542030BD012901D00229E4D1818F01F2B9
:1068A00033318187E8E703F11402914203DD1439A3
:1068B000A0F8541030BDA0F8543030BDFC060020C4
:1068C00014000020F30600209C020020B6040020E3
:1068D000B4040020B0040020400100202005002066
:1068E000B80400202DE9FC4101210220FDF7DCFA6B
:1068F00001211920FDF7F0FA01213C48FBF7C8FC03
:106900004027ADF8007003248DF802400420384D74
:106910008DF8030069462846FBF768FCE001ADF8F6
:1069200000008DF802401C208DF8030069462846BF
:10693000FBF75CFC4FF4E0712846FBF7DEFCA81582
:10694000ADF800008DF8024010208DF80300694674
:106950002848FBF74BFC4FF4A060FCF7AFFF1D206D
:106960008DF8040001268DF8056000258DF806508D
:106970008DF8076001A8FCF76FFF1F498C20088085
:106980001D494FF6FA702C3108806E20091F0880CF
:1069900019481430068018480830078016492031FD
:1069A0000D80154AD020121D1080134A45F2F300C5
:1069B000183210800A1F45F2500010800E4A4FF620
:1069C000FF7038321080121D1080121D108041F2AD
:1069D0001B10088000F012F8FBF70CFF064810307F
:1069E0000580001F0480BDE8FC810000000C1A0037
:1069F00000100140000C01400004004070B51D2053
:106A0000FCF7FEFE2A4D40212846FBF76DFC840072
:106A100080212846FBF768FC44EA4004A915284673
:106A2000FBF762FC0443E0B2224C84F83C00FBF725
:106A3000E7FC0546052805D91F48C18841F04001FB
:106A4000C18001E084F838501C48007A000703D563
:106A500094F838001A490D5C4FF6FA702063E06232
:106A6000A06260622062E061A0611648606300205D
:106A70006064A06484F83F0084F84000FBF76EFC7B
:106A8000A07AFF2811D0022084F83D000E4800882B
:106A900020662846FCF710F9207820F001002070CD
:106AA000BDE870401D20FCF7C1BE0120ECE70000EE
:106AB00000100140400100200C0A00209C02002030
:106AC0003C920008DCFF0500240400402DE9F0435F
:106AD0004E484F4902880B889A1A92B20F2A69D3FE
:106AE000098801804B49098B027D00EB42029180AD
:106AF000017D491CC9B2017508295BD300240475C6
:106B00002246017D00EB4103491CB3F90430C9B2B0
:106B100002EB630212B201750829F2D33E490475F3
:106B20003E4B4A8044800E789D895FEAC67C40F6E1
:106B300038694FF0030714D0A2F22B5C42F6E858F4
:106B4000C44520D3A1F1020C26F00204ACF80020C9
:106B500047750C7040F22B54A24211DA45F0040242
:106B60001EE046F001060E704A4507DD45F00102C1
:106B70009A8126F002020A70477519E0447517E001
:106B800045F002020CE04A450CDA8775427D12B1ED
:106B9000521E42750CE046F002020A7025F0070210
:106BA0009A8105E0B30703D5837D2BB15B1E837506
:106BB00040888880BDE8F08342F6AA239A4222DA10
:106BC000B1F904302BB941F2CD05AA4201DA448073
:106BD000EEE7134C920302EB843241F67244B2FBAF
:106BE000F4F214B240F2333502464480AC4200DA8B
:106BF0005580B2F90240E41A04F5A374B4F5237F7A
:106C0000D6D84380D4E74FF48043FAE7940A0020B3
:106C1000FC0600209C020020CA0500200C0A00206F
:106C2000C8F1FFFF2DE9F0416C4CDFF8B4E14FF003
:106C3000000594F82810C80706D094F92C104B4290
:106C4000002956DD0E4655E0664884F82B50E5864F
:106C5000654A90F8380084F834001586CEF8045060
:106C6000CEF80850614E40F26663CEF80C50A4F89E
:106C7000703036F810005E4E768830444FF6FF765E
:106C800006EA800024F8240B4FF080602060A320E7
:106C9000208460845810A084E38440F699102085F5
:106CA000580060854FF48050A08541F23330E08574
:106CB00041F26660208641F69910608641F6CC402C
:106CC000A0864FF40050E08642F23330208742F233
:106CD0006660608742F69910A08742F6CC40E08754
:106CE00082F89D5041F00100207184F84450BDE8C5
:106CF000F0811E4694F92B004242002801DD074630
:106D000000E01746F61B012E0BD0002800DB0246E0
:106D10005FFA82F684F82C0094F84300012805D02D
:106D200041E0002900DA1946CEB2F3E794F92D309C
:106D30005942002B01DB184600E0084694F92E204A
:106D4000C7B25042002A01DB944600E08446BC45AD
:106D500008DD002A00DA0246D7B2002B00DA0B4623
:106D6000D8B207E0002B00DA0B46DFB2002A00DBC6
:106D70001046C0B204EB4000B0F9441004EB4700E9
:106D800030F9442F11444910018084F8435084F8AD
:106D9000325084F8315084F8305084F82F5084F801
:106DA0002E5084F82D5004EB46007546B0F944008F
:106DB000E086BEF80410C82309B26422FDF780FD06
:106DC0006860E968401AA9680844A860B5F900102D
:106DD0004843C013E860A4F8700088E7200A002048
:106DE000B8050020400100209C0200204E920008BF
:106DF000600000202DE9F0415F4C94F82800C007A6
:106E000079D05E4894F83410002690F838005C4D34
:106E1000814271D05B4AA4F866605B4F535C2246A6
:106E2000834292F92B2002D07B5C83420FD1521C0B
:106E300052B284F82B20795C814202D1521C84F832
:106E40002B2094F92B100F291BDD0F2117E04F4B3E
:106E50005F5C4F4B874202D05F5C874211D1521E6C
:106E600052B284F82B20595C814202D1521E84F820
:106E70002B2094F92B206FF00E018A4201DA84F85E
:106E80002B103D4994F833302D3194F82B205A546F
:106E900094F83310491CC9B284F83310062901D381
:106EA00084F8336094F92D2094F92F108A4211D17F
:106EB00094F9312091420DD194F92E2094F930109B
:106EC0008A4207D194F93220914203D1012184F8FA
:106ED000431001E084F84360284984F8340094F9B1
:106EE0002B300978012B0DDD254A4F07926804D518
:106EF00042F0080203E03CE015E022F00802AA603C
:106F000084F82900B3F1FF3F0ADA4907A96802D5DE
:106F100021F0080101E041F00801A96084F829008E
:106F2000FBF71CFA11E094F8430001280DD1B4F8E6
:106F3000660043F60951401C80B2A4F866008842FE
:106F400003D9A4F8666084F84360E87B082810D071
:106F5000B5F93010512341220020FDF7B1FC2886FD
:106F6000002806D10B48067014F8280F20F0010005
:106F70002070BDE8F0810000200A002040010020C0
:106F80009C020020309200083692000842920008CD
:106F900048920008F306002030B52049204AB1F895
:106FA0006A301088C01A80B20F2836D31088A1F832
:106FB0006A001C4D00204FF000432A5C940903D066
:106FC0000124B4EB921F24D1D20622D0164A52F8E3
:106FD00020201268134C123434F81040224201EB86
:106FE000000494F9722008D00A2A04DB0A6823FA04
:106FF00000F4224308E0521C09E012F10A0F05DCFC
:107000000A6823FA00F4A2430A6002E0521E84F8E0
:107010007220401CC0B21128CFD330BDD005002053
:10702000FC0600203C8E00083C8F00082DE9F0078C
:1070300079497A480A8903889A1A92B2082A74D33D
:1070400000880881A1F12C0042890AB1521E4281B8
:10705000734A92F82820802A67D302F03F020A7010
:10706000C2890AB1521EC281B1F90620902A0CDBF6
:107070008A46FF2A09D08146C089002855D169482F
:1070800000230078092805D005E0BDE8F007624834
:1070900000F092B90823644A92F8EA500DB143F027
:1070A00004036248817AC90701D043F00203D2F891
:1070B00008C05FEA0C5101D543F0010317680021B5
:1070C0005B4EFC0302D596F8654004B18021C4886C
:1070D0005FEA446801D541F040015FEA845801D578
:1070E00041F020015FEAC47801D041F01001007A3C
:1070F000400701D541F008014E480078C00701D093
:1071000041F00401A00601D541F001010020012D4C
:1071100000D1082096F8705085B992F84620022ACE
:1071200004D0012A05D03AB108E072E040F0030033
:1071300004E040F0020001E040F001007A0701D4D1
:1071400040F02000CCF3C0020025CCF3002C6245B7
:1071500002D13A0700D4042596F86F20012A01D104
:1071600045F00105344A0027BC4612783E46C2F37A
:107170008102012A04D0022A04D0032A04D004E0A8
:10718000022602E0042600E010262C4A64060ED5F2
:10719000214C1C342478240609D51478640606D4BE
:1071A000274A40F6CC44926D6243140C05E0B2F8D5
:1071B000AE2040F699146243940B4FF008088AF809
:1071C0000A804FF061088AF80B808AF80C308AF840
:1071D0000D108AF80E008AF80F508AF81070270AEE
:1071E0004B4083F06901414069408AF81170794051
:1071F0008AF81240614052468AF813C071408AF8FA
:10720000146051754FF4C871A9F80E10FF20AAF848
:107210000600BDE8F0077047B8060020FC06002015
:10722000D0050020F30600209C0200200C0A00205C
:10723000600C002004090020B80400204001002058
:10724000EC0700204C48816941F0FC0181614FF45A
:10725000A060FCF733FBFBF75BFBFCF79BFCF9F74B
:10726000A7FCFCF789FAFDF731FAFFF73BFBFCF7C7
:10727000C9F9FFF7C3FBFBF7BDFA404D4FF40050CF
:10728000A5F81601FEF7E4FD00214FF4FA5340F291
:10729000EE220020401C80B29842FBD3491C89B2E8
:1072A0009142F6D33648002680F87260F9F716FB53
:1072B000F9F7B8FFFCF79EFCF9F786FEFEF7BEFE75
:1072C000102230493048F8F760FF304C314FE088E9
:1072D00020F04000E0802E48017821F0200101706C
:1072E000FA20F8814FF49670E887FFF701FA2A49EF
:1072F0002A48FCF7F5FB2A48FCF71EFC2948416A9E
:1073000088472948416B8847FEF7ECFF2749422010
:10731000C8802749C8603E71E088E08120892082CA
:1073200060896082FAF7DAFEFAF73CFEFFF776F83A
:10733000FFF7CCFB00F0F8F9FFF72EFE00F0C2FFDC
:10734000FEF710FAFAF792FCFBF7D4FCFFF72CFAE1
:10735000FCF7A8FEFBF7F6F8FBF728F900F07AF83F
:10736000FFF764FE1348FAF779FA00F06FFAFDF7B9
:10737000F1F9FAF7DDFBCFE7001002409C02002094
:1073800020050020600C0020100600200C0A0020C0
:1073900040010020F00600208C0800206808002032
:1073A000FC03002034000020D0000020180700203B
:1073B0002C0400208C090020F0B523490278B0F994
:1073C000064000231F4E31F81210FF2C18D0B0F9E0
:1073D00004701E4DBC4231DA00EBE40704F00704F0
:1073E000BF7AA7408478FFB23CB190F801C0ACF1FD
:1073F000010C64451FDA3C061DD455F822200DE02F
:1074000056F82220116012498A79521CD2B28A7130
:10741000022A02D38370C3808B71F0BD1160817822
:10742000491CC9B2817042789142F6D38370C188F9
:10743000491CC180F0BD56F82220EFE755F8222004
:107440001160F4E71C9000084E8E0008C48F0008FD
:107450008C060020F0B561486149B0F86C200B88BB
:107460009A1A92B29C2A7BD30988A0F86C105D49C5
:107470005D4F91F82A1001F0070297F84610022A92
:1074800000D1491E594C80F83E104FF00203E288AB
:107490004FF00001550401D5012236E0A489E5062C
:1074A00001D5062231E0250701D508222DE0550639
:1074B00003D44F4D2D78AD0601D5042225E01505E6
:1074C00001D5072221E0150601D50A221DE0950607
:1074D00001D50C2219E0150701D50B2215E055073F
:1074E00001D4D50501D510220FE0D50601D505221E
:1074F0000BE0650703D4A50701D4E40702D080F8A8
:107500006E3007E0920403D5032280F86E2001E07C
:1075100080F86E10374A384C92F820E0324A251F26
:10752000D2F808C02D4AB2F87060721C92B2BEF157
:10753000000F0DD02CF4000CC7F808C090F86E7046
:10754000B7B11E2F1AD090F86F200AB325E007E0DC
:107550004CF40006BE60A0F870200A2A01D2236015
:10756000F0BD142A01D22B60F0BDA0F87010F0BD60
:107570002B60A0F8701080F86F10F0BD642E04D25C
:10758000A0F87020322AEED3E9E7A0F87010EAE7FD
:107590007F1C80F86F70A0F8701090F86F20012A9F
:1075A00010D0002AE9D0B0F87060761CB6B2A0F80E
:1075B00070601E2ED7D323603C2EDED9521E80F879
:1075C0006F20D2E7B0F87020521C92B2A0F8702061
:1075D0002360C82AD1D980F86F10C6E7D0050020F3
:1075E000FC060020600C00209C0200200C0A0020F9
:1075F00040010020B8040020141C0140F0B54248AE
:10760000B0F84810491C89B2A0F8481002297AD372
:107610003E490024A0F848400A783D4B042A57D040
:107620004FF48041082A0BD0A0F10C02B2F90020DF
:107630008A4200DA1146B3F980208A4200DA114604
:10764000344A92698A4200DA11B2418282881D8AE4
:10765000C2EB8502304D12B22D78C5F381062A4D5A
:1076600042F2AA467243B5F9765092126A43121357
:10767000C26086681546C6EBC60642F3D102F60222
:1076800002EBA6328260C66C1644C664B0F8507035
:107690007F1CBFB2A0F85070B7F5806F04D3B6124C
:1076A0000682A0F85040C464891A1C4EC26A724314
:1076B00040F255564E4302EB4602466A324442625D
:1076C000B3F93030B2EB034F06DD1A04426206E034
:1076D0001349B1F90410B3E7002A00DA4462C16229
:1076E000104990F83D2091F838108A420BD080F86C
:1076F0003D10B0F84210A0F84410B0F84010A0F8C7
:107700004210A0F84050F0BD20050020F3060020F4
:107710009C020020F80B0020B8040020C3F5FFFFF6
:10772000140C00204001002017481849B0F85A20D6
:107730000B889A1A92B20F2A25D30988A0F85A10FA
:10774000134941F6515391F84D10CA0701464FF4C1
:107750008042B1F9001059438913A0F86C100D490B
:107760000B78A0F10C01022B06D1B1F90030934245
:1077700002DA1B1D0B8000E00A800021A0F86010D7
:1077800020F85C1F4280704720050020FC06002086
:10779000600C0020F30600204FF6FF7202EA800220
:1077A00010F4404315480ED0B3F5804F14D0B3F514
:1077B000004F4FEA122216D0C2F5807330F8133012
:1077C0005B424B8005E0120A30F812304B80C2F564
:1077D000807230F812000FE0120AC2F5807330F8A0
:1077E00013304B8005E030F81230C2F580725B42F6
:1077F0004B8030F81200404208807047388C0008F7
:10780000104A518A908AD28A16384639A2F111025A
:1078100000D54942002A00DA52421144002800DA19
:1078200040420844084943F6284300B2B1F93620E3
:107830005A43921340F2D733584302EBA030C88624
:10784000704700009C02002020050020F0B5904900
:1078500090480A8903889A1A92B23E2A1ED3008859
:10786000088101F138004FF4FA63428A9A4202D249
:10787000521C428200E04382874A92F82220802AEA
:107880000CD302F03F020A70B1F90620402A06DB51
:10789000FF2A04D0C2883AB1521EC280F0BDBDE8B2
:1078A000F0407B48FFF788BD428A9A42F6D30778BA
:1078B0004FF0010E3A074FF0FF055BD5847A40F296
:1078C000DC52630708D444F004038372C28081F859
:1078D0000BE081F80AE04CE04378072B05D0032B3E
:1078E00003D0052B01D0062B07D1660605D444F042
:1078F00040038372C280052239E0654A5FEA437C17
:1079000002F138024FF42076127A0DD55FEAC26C8C
:107910000AD45FEA446C07D442F0100202723A06BD
:1079200028D4C680192222E0DF0709D0970707D4A0
:10793000670605D442F002020272C680042216E0F5
:107940009F0709D5170707D4670605D442F0080238
:107950000272C68003220AE01B070BD5530709D425
:10796000630607D442F004020272C6800B22CA7278
:107970008A72CD80494AB2F92230B2F91A7003F204
:107980003D140022A74200DB0276414E444C06F132
:107990003806A479B6895FEAC46C06F101064FF493
:1079A000C874B6B213D58681B6F57A7F05D9017A47
:1079B00021F0800101728281F0BD037A1E06FBD4A2
:1079C000828143F080020272C480112035E09F4220
:1079D00016DA037E052B13D28681B6F5487F04D9CB
:1079E0008281027A22F040020272027A5606E3D4C1
:1079F0005B1C037642F040020272C48002201CE04D
:107A0000284B1C89C4F3C006C4F3002740F2EE24BF
:107A1000BE4216D11E78360713D4427E012ACBD13E
:107A2000428BB2F5167F02D2521C4283F0BD827A9D
:107A300042F002028272C4800F20C8728872CD8028
:107A4000F0BD93F80D714FF40046012F18D1164F79
:107A500041F6583C7F6C674512DD83F80CE1134B0F
:107A60001E60C38AA34202D25B1CC382F0BD4FF4E6
:107A7000FA73C3801C23CB728B72CD80C282F0BD9F
:107A8000C2820A4883F80C21001F0660F0BD000086
:107A90009C060020FC060020D0050020B804002031
:107AA0000C0A00209C020020400100201408014024
:107AB0002DE9F05FFB48FC49DFF8F0A3007E0A1DCA
:107AC000131D0128504658D030F85A4F0C80418879
:107AD0001180BAF85E001880F54DF64C49F2CD32AF
:107AE000B5F91E006083B5F9201043F6CC4C00EBCD
:107AF000410151430914A183B4F92230B4F9206043
:107B000001FB03F200FB062242F38F326282B4F9DA
:107B1000167007FB0CF7BF1340F2333C714302FBB6
:107B20000CF200FB131007EBA232E28240F38F301D
:107B3000A082B4F91810E04FC1EBC10141F3D101AB
:107B400001EBE000DD4E2083786C30603169304617
:107B50008847DB49308948800846FDF735FFDFF864
:107B6000649301264FF0000B99F8000008280CD010
:107B7000618E218204284AD01AE030F8604F0C80D0
:107B800041881180BAF86400A5E7CF4890F92B101E
:107B9000491C022939D890F8681019B1B4F852007C
:107BA000208205E0618E2182A4F8521080F868607E
:107BB000B4F91410B4F90A00C44AF9F76DFCE06294
:107BC000BAF91611884204DDC048E162027A914098
:107BD0000162B848DFF8F8E24C3847F2A3080278AF
:107BE0004EF2461172B3012A52D080F800B000BFA5
:107BF00099F8000004280DD0B44AB4F91210B4F971
:107C00000800243AF9F748FC07E0608EC8E7686A84
:107C10000014E062B87A70B3AE48AF4DA06228603D
:107C2000E06A68602846FCF7A3F8A84F287C383F34
:107C300001285ED0A06A3860A8480178C9075CD0E6
:107C400040695BE0B5F91E2042448A4209D8B5F983
:107C5000202042448A4204D8B5F9222042448A4274
:107C6000C6D9A0F802B0B7F8AE205946B2F5C87F21
:107C700002D8467007E039E0B2F5487F01D8022209
:107C800000E0032242708AF80F1089F8001024E007
:107C900080F800B0B5F91EC05A46C4448C4509D8D6
:107CA000B5F920C0C4448C4504D8B5F922504544E8
:107CB0008D429DD9B7F8AE10B1F5C87F01D8467096
:107CC00006E0B1F5487F01D8022100E003214170B0
:107CD00042808AF80F2089F80020BEF8061041F48F
:107CE0000061AEF80610FAF74FF981E74FF4AF7074
:107CF00093E768693860A86900E0E06A78607348D3
:107D00003838FCF7A9F96B4D6A4935F8100F3C3942
:107D1000FFF742FDDFF89C91DFF8C481A9F14C091F
:107D2000D9F81010C9F86C10B5F91010B868B5F989
:107D3000122000FB01F4FB68504303FB124444F3A0
:107D40008F3703FB010040F38F34AF86EC86A8F831
:107D500002704546A8F804404046FEF7E1F9287F46
:107D600009F11405012830D0604241104DF6B3509E
:107D700047433A1469802A808B18A9F80440A9F86F
:107D80000630891AA9F808108AF80CB0B9F904303D
:107D9000D84654464946002B00DD2673B1F906004B
:107DA000002802DD227B921C2273B9F90820002AE8
:107DB00002DD217B091D2173217B072920D2DFE809
:107DC00001F01F1B3419301D3200B8F920304DF678
:107DD000B352584240106880B8F91E10514309143C
:107DE0002980A9F804304318A9F80630401AA9F8E8
:107DF0000800C9E7667303E0022100E00321617314
:107E0000DFF8B090374E384F99F800100129617BA8
:107E10000DD0072945D2DFE801F0E7FEFDFCFBFAB3
:107E2000F9000421EBE70521E9E70621E7E7072947
:107E300037D2DFE801F0D9041B627999AF0001461F
:107E40001846FBF733FE2860B5F90200B5F90010BB
:107E500043F2046201445143090C5043A4F85A1000
:107E6000000CA4F85C00A4F85E8027E1404201B257
:107E7000504200B2FBF71AFE2860B5F9020043F247
:107E800004614143090CA4F85A10B5F900100844E4
:107E900043F204614843000CA4F85C00A4F85E803F
:107EA0003AE1A1E08C090020342C01409C02002022
:107EB0002005002060000020400100202C0400204C
:107EC000EC030020F3060020200A00208C0800208C
:107ED0000C0A0020A2FEFFFFE40900200409002094
:107EE000C009002000240140002801403046F8F776
:107EF000BDFE01231A4607216BE019461046FBF729
:107F0000D5FD2860A4F85A80B5F90200B5F9001033
:107F100043F2046201445143090C5043A4F85C103D
:107F2000000CA4F85E0026E15942404209B200B2BA
:107F3000FBF7BCFD2860A4F85A80B5F9020043F2B3
:107F400004614143090CA4F85C10B5F90010084421
:107F500043F204614843000C39E13046F8F786FEED
:107F600001231A46052134E01146FBF79FFD2860E6
:107F7000B5F9020043F204614143090CA4F85A1018
:107F8000A4F85C80B5F90010084443F2046148434A
:107F9000000C47E1504201B2584200B2FBF786FDA7
:107FA0002860B5F90200B5F9001043F204620144FB
:107FB0005143090CA4F85A105043A4F85C80000CFB
:107FC000A4F85E005EE13046F8F750FE01231A4641
:107FD00006213846F8F74AFE01213046F8F7BCFD85
:107FE00001213846F8F7B8FDB34EB9F808004D4600
:107FF0003080B9F80A007080B9F81000B0803046BF
:10800000F9F778FCB4F85A00F18805E018E1ECE0E3
:10801000BDE08EE05EE031E00844A4F86000B4F812
:108020005C0031890844A4F86200B4F85E007189EC
:108030000844A4F86400317EA048012978D034F8BF
:108040005A1F018061884180A18881809B490288F4
:1080500008310A8042884A80808888809748896AE7
:108060000830884795F8360000287DD0F8F7FEFFE5
:1080700015F8360F401E2870BDE8F09F01461846DF
:10808000FBF714FD2860B5F9020040F68151484322
:1080900080136880B5F9001040F68152514389136E
:1080A0004218A2F68152524252082980A4F85E205A
:1080B0001044A4F85C000844A4F85A00002130469B
:1080C000F8F74AFD00213846F8F746FD01231A4625
:1080D00006210BE7404201B2504200B2FBF7E6FC3A
:1080E0002860B5F9020040F681514843801368804A
:1080F000B5F9001040F68152514389134218A2F697
:108100008152524252082980A4F85E201044A4F8FB
:108110005A000844A4F85C0000213046F8F71CFD22
:1081200000213846F8F718FD01231A460521DDE63F
:10813000B4E019461046FBF7B9FC2860B5F9020017
:1081400040F68151484380136880B5F9001040F62D
:108150008152514389134218A2F68152524229801A
:108160005208A4F85A2000E09BE01044A4F85E00F6
:108170000844A4F85C0000213046F8F7EDFC00212B
:108180003846F8F7E9FC01231A460721E5E659428B
:10819000404209B200B2FBF789FC2860B5F9020041
:1081A00040F68151484380136880B5F9001040F6CD
:1081B0008152514389134218A2F681525242520809
:1081C0002980A4F85A201044A4F85C000844A4F8BC
:1081D0005E0000213046F8F7BFFC00213846F8F772
:1081E000BBFC01231A460621B7E61146FBF75EFCED
:1081F0002860B5F9020040F6815148438013688039
:10820000B5F9001040F68152514389134218A2F685
:108210008152524252082980A4F85C201044A4F8EC
:108220005A000844A4F85E0000213046F8F794FC98
:1082300000213846F8F790FC01231A460521C2E6D2
:10824000504201B2584200B2FBF730FC2860B5F949
:10825000020040F68151484380136880B5F9001050
:1082600040F68152514389134218A2F6815252427C
:1082700052082980A4F85C201044A4F85E00084449
:10828000A4F85A0000213046F8F766FC0021384671
:10829000F8F762FC01231A46072194E634F8601FC0
:1082A000CFE607480088A0F5D04168393FF4E4AE36
:1082B000BDE8F05FF9F7AEBD8C0900202C0000206E
:1082C000182C01402DE9F041904C9148B4F85A1017
:1082D0000288511A89B20F296FD30088A4F85A0076
:1082E0008C480088DFF83082C0074FF000054FF05F
:1082F000010741D0874AD4E90C1024321388B1EB2E
:10830000530F02D21288511A08444FF4F371884275
:1083100000D208468149B1FBF0F0616CC1F3510114
:10832000084406466064F8F77AF800227C4BF7F7B9
:10833000E2FF4FF040427B4BF7F7DDFF0E22F8F7EC
:1083400049F8F8F7A3F8A4F8A40094F86500401CD5
:10835000C0B284F86500082834D36C4898F84620E9
:10836000001F03789A4201D0027045806E4A13784C
:108370006E4A23B1458021E06564A56458E0D8F8D1
:108380009410A1F5FA618E4211DD616D8B1C9E4245
:1083900005DDB0F902100A290DDA491C06E08E420B
:1083A00005DAB0F90210002908DD491E4180B0F954
:1083B00002000A2802DB177001E0A2E01570666572
:1083C00084F865505A484FF4A5420178C1F3810101
:1083D000012949D002294AD044F687712181A4F8A5
:1083E000A020B0F9243089B24B439B13A4F89C30F1
:1083F000B0F90E0000237043B0FBF1F0A16CC0F3A4
:10840000D100C1EBC101C90200EB9130A064F017AB
:10841000810341EA9641B003F7F786FEB4F8A21053
:10842000C1EBC101C902C00800EB9130A4F8A20061
:10843000616CA06E0844A06694F86C20521CD2B205
:1084400084F86C20082A05D3C008A4F86E0084F8CC
:108450006C50A566374A384ED388580633D498F8FE
:108460000F00022806D02CE043F20451B6E744F294
:108470004621B3E7B06840F69916B04221DD94F882
:10848000380094F88660B0420CD084F8860094F8E6
:108490003D0000F00106C0F34000864202D1A4F87E
:1084A000825004E0B4F88200B0F5966F05D2B4F8BB
:1084B0008200401CA4F8820005E043F08000D080D8
:1084C00001E0A4F88250114894F83F20B0300C2A03
:1084D00001D2C57400E0C774174B41F2482641F23F
:1084E000504C93F83C400C4B0C2AB3F882300AD322
:1084F000B14208DB012C06D0614502DD002B00D122
:108500008774BDE8F0818574FBE70000400100201E
:10851000FC060020000400409C0200204564BD01D0
:1085200000209C40133B3340EA030020EB03002073
:10853000B80400200C0A0020200500202DE9F0419D
:10854000384C394E394F207841F23331C2074FF061
:1085500000050CD0A28962B394F90700002800DA64
:108560004042C0B2032829D240F2AE702AE0A57082
:10857000E5732F4AE571A58192F83830237220F017
:108580000800A18040F0020020703D867560B56053
:10859000F560916C490005D041F68461A18140F0FD
:1085A00010002070C0B240F0010020706574BDE87A
:1085B000F081658120F01000207015E0042803D2BE
:1085C00040F6510060810FE0052802D240F6991074
:1085D000F8E740F6CC42062803D3072801D3082841
:1085E00001D2628100E0618197F89D0098B9B0885E
:1085F000102301B2B4F90A003622FCF761F9706069
:10860000F168401AB1680844B060B6F900104843F8
:10861000C013F0603886388E10B10120A070C6E714
:10862000A570C4E7140C00207C0600209C020020EA
:10863000400100202DE9F041554C2678F0077CD010
:108640005448217A544D90F8380081427BD0534AE7
:108650002346DFF84CC1575C93F90E2093F907309D
:10866000874203D01CF80170874213D146F00206FE
:108670005B1C26705BB2E3711CF80110814201D1D2
:108680005B1CE37194F90710062901DD0621E171F5
:10869000521C1CE0434F17F801C0434F844503D0E0
:1086A00017F801C0844513D126F002065B1E267020
:1086B0005BB2E371795C814201D15B1EE37194F995
:1086C00007306FF005018B4200DAE171521EA27390
:1086D000207294F907108A1C042A02D941F6846298
:1086E000A2812C4A012912780ADD2B4B56079B6880
:1086F00002D543F0080301E023F00803AB6060708B
:10870000B1F1FF3F09DA5107A96802D521F008014C
:1087100001E041F00801A9606070F9F71FFEA07840
:10872000012810D121488068A3280CDA94F90700A9
:10873000022803DD0220E07105E01EE06FF0010178
:10874000884200DAE171A089002630B1401E0004A1
:10875000000CA08101D1E671A673E87B04280CD03F
:10876000B5F93010512341220020FCF7A9F82886E2
:10877000002802D1E07B10B1A670BDE8F0810C4862
:1087800006700C480670207820F001002070F4E795
:10879000140C0020400100209C02002030920008B0
:1087A00036920008429200084892000820050020F6
:1087B00010070020F3060020743F713D9B3BED390C
:1087C0006238F436A13565343F332A3227313330ED
:1087D0004C2F722EA32DDF2C242C722B0000003680
:1087E000220200388E03003AB005003C1C07003E10
:1087F00088080040F4090042AA0A0044160C00460A
:10880000CC0C0048820D004A380E004C00000036A7
:10881000220200388E03003AB005003C1C07003EDF
:108820001C0700401C0700421C0700441C070046B0
:108830001C0700481C07004A1C07004C00000036BB
:10884000220200388E03003AB005003C1C07003EAF
:1088500088080040F4090042AA0A0044160C0046A9
:10886000CC0C0048820D004A380E004C0000003647
:10887000B60000382202003A8E03003CFA04003EA3
:10888000660600401C070042D207004488080046E4
:10889000880800488808004A8808004C000000400A
:1088A00022020044440400486606004C3E09005081
:1088B000160C0054EE0E0058C711005C9F140060A7
:1088C000771700644F1A0068271D006C00000040F5
:1088D000220200448E030048B005004C1C070050E3
:1088E00088080054F4090058600B005CCC0C006050
:1088F000380E0064380E0068380E006C000000402E
:1089000000000044000000480000004C000000503F
:1089100000000054000000580000005C00000060EF
:1089200000000064000000680000006C4414585807
:1089300058701111585858704111585848701114F6
:1089400048585870141158485870E8190056E819DA
:108950000054E8190052E8190050E819004EE819CF
:10896000004CE819004A1E1A00482C1B0046011D45
:108970000044B51D00429C1F0040EE21003EF9233B
:10898000003C1626003A5E260038DC2600363228E7
:10899000003441290032152B0030242C002E7A2D72
:1089A000002CF42E002A11310028683200263C34B5
:1089B0000024113600221B3800204A3A001EE53CF4
:1089C000001C0040001A0040001800400016004043
:1089D000001400400012004000100040000E004053
:1089E000000C0040000A0040000800400006004063
:1089F00000040040000200400000000001020304E7
:108A00000500050001020304010400030502000043
:108A1000F001000036010000F8000000BA0000007C
:108A20007C0000007C0000007C0000004114141158
:108A300011144411141441110000290052007B004C
:108A4000A400CC00F5001E01470170019901C2018C
:108A5000EA0113023C0265028E02B602DF0208033D
:108A6000300359038203AA03D303FB0324044C04F9
:108A700075049D04C504EE0416053E0567058F05C3
:108A8000B705DF0507062F0657067F06A706CE06A1
:108A9000F6061E0746076D079507BC07E4070B0897
:108AA000320859088108A808CF08F6081D094409AA
:108AB0006A099109B809DE09050A2B0A520A780ADF
:108AC0009E0AC40AEA0A100B360B5C0B820BA80B39
:108AD000CD0BF30B180C3E0C630C880CAD0CD20CB8
:108AE000F70C1C0D410D650D8A0DAF0DD30DF70D63
:108AF0001C0E400E640E880EAC0ECF0EF30E170F38
:108B00003A0F5E0F810FA40FC70FEA0F0D10301040
:108B1000531075109810BA10DD10FF102111431179
:108B200065118711A911CA11EC110D122E125012E4
:108B300071129212B312D412F41215133613561383
:108B400076139613B713D713F61316143614561458
:108B500075149414B414D314F214111530154E1561
:108B60006D158C15AA15C815E7150516231641169F
:108B70005F167C169A16B716D516F2160F172C1715
:108B8000491766178317A017BC17D917F5171118BF
:108B90002E184A18661881189D18B918D418F0189C
:108BA0000B19261942195D1978199219AD19C819AE
:108BB000E219FD19171A311A4C1A661A801A991AF5
:108BC000B31ACD1AE61A001B191B331B4C1B651B6D
:108BD0007E1B971BAF1BC81BE11BF91B121C2A1C19
:108BE000421C5A1C721C8A1CA21CBA1CD21CE91CF6
:108BF000011D181D301D471D5E1D751D8C1DA31DFB
:108C0000BA1DD01DE71DFD1D141E2A1E401E571E35
:108C10006D1E831E981EAE1EC41EDA1EEF1E051F9B
:108C20001A1F2F1F451F5A1F6F1F841F991FAE1F2A
:108C3000C21FD71FEC1F002000006400C9002D01D7
:108C40009201F7015B02C00224038903ED03520481
:108C5000B6041A057F05E3054706AB060F07730741
:108C6000D7073B089F0802096609C9092D0A900A1F
:108C7000F30A560BB90B1C0C7F0CE20C440DA60D2D
:108C8000090E6B0ECD0E2F0F900FF20F5310B41074
:108C900015117611D71138129812F8125813B8130B
:108CA00018147714D61435159415F3155116B016FB
:108CB0000E176B17C91726188318E0183D19991954
:108CC000F519511AAD1A081B631BBE1B181C731C27
:108CD000CD1C261D801DD91D321E8A1EE31E3B1F82
:108CE000921FEA1F41209820EE2044219A21EF2173
:108CF00045229922EE2242239623E9233C248F2405
:108D0000E22434258525D72528267826C826182745
:108D10006827B72706285428A228EF283D29892943
:108D2000D629222A6D2AB82A032B4D2B972BE12B0B
:108D30002A2C722CBB2C022D4A2D912DD72D1D2EA5
:108D4000632EA82EEC2E302F742FB82FFA2F3D3023
:108D50007F30C030013141318131C13100323F3289
:108D60007D32BA32F73234337033AC33E7332234E6
:108D70005C349534CE3407353F357735AE35E43540
:108D80001A3650368536B936ED36203753378637A2
:108D9000B737E937193849387938A838D738053915
:108DA00032395F398B39B739E2390D3A373A603A9F
:108DB000893AB23ADA3A013B283B4E3B733B983B47
:108DC000BD3BE03B043C263C483C6A3C8B3CAB3C16
:108DD000CB3CEA3C093D273D443D613D7D3D993D0D
:108DE000B43DCE3DE83D013E1A3E323E493E603E36
:108DF000763E8C3EA13EB53EC93EDC3EEF3E013F95
:108E0000123F233F333F433F513F603F6E3F7B3F25
:108E1000873F933F9E3FA93FB33FBC3FC53FCD3FF8
:108E2000D53FDC3FE23FE83FED3FF13FF53FF93F03
:108E3000FB3FFD3FFF3FFF3FFF3F0000E7382C3582
:108E4000002020EF2037202333202620210000801F
:108E500002000400080010000002000400080400E2
:108E60000002000400080010002000400080040000
:108E70000000008000000040000000200000001002
:108E800000000008000000040000000200000001D3
:108E900000008000000040000000200000001000E2
:108EA00000000800000004000000020000000100B3
:108EB0000080000000080140000C0140000C01404F
:108EC000000C0140000C0140000C0140000C01406E
:108ED000000C014000100140001001400010014052
:108EE000001001400010014000100140001001403E
:108EF000001001400014014004080140040C01402E
:108F0000040C0140040C0140040C0140040C01401D
:108F1000040C0140040C0140041001400410014005
:108F200004100140041001400410014004100140ED
:108F300004100140041001400414014008080140DD
:108F4000080C0140080C0140080C0140080C0140CD
:108F5000080C0140080C0140080C014008100140B9
:108F6000081001400810014008100140081001409D
:108F70000810014008100140081001400814014089
:108F80000C0801400C0C01400C0C01400C0C014081
:108F90000C0C01400C0C01400C0C01400C0C01406D
:108FA0000C1001400C1001400C1001400C1001404D
:108FB0000C1001400C1001400C1001400C1001403D
:108FC0000C14014010080140100C0140100C01402D
:108FD000100C0140100C0140100C0140100C01401D
:108FE000100C014010100140101001401010014001
:108FF00010100140101001401010014010100140ED
:10900000101001401014014000000000000000009A
:1090100000000000000000000000000014080140F3
:10902000140C0140140C0140140C0140140C0140BC
:10903000140C0140140C0140140C014014100140A8
:10904000141001401410014014100140141001408C
:109050001410014014100140141001401414014078
:109060000000000000000000000000000000000000
:1090700000000000FFFFFF0F0FFFFFFFFFF0FFFFEB
:10908000FF0FFFFFFFFFF0FF0FFFFFFFFFF0FFFFEE
:10909000FF0FFFFFFFF0FFFF0FFFFFFFFFF0FFFFDE
:1090A000FF0FFFFFFFFFF0FFFFFF0FFFFFFFFFF0CE
:1090B000FFFFFF0FFFF0FFFF000000404000000037
:1090C0000004000000400000000004004000000018
:1090D0000004000000400000000400004000000008
:1090E00000040000004000000000040000004000F8
:1090F00000000004000000400004000000000080A8
:10910000800000000008000000800000000008004F
:10911000800000000008000000800000000800003F
:10912000800000000008000000800000000008002F
:10913000000080000000000800000080000800001F
:1091400000000020200000000002000000200000BD
:1091500000000200200000000002000000200000CB
:1091600000020000200000000002000000200000BB
:1091700000000200000020000000000200000020AB
:109180000002000000000060600000000006000017
:109190000060000000000600600000000006000003
:1091A00000600000000600006000000000060000F3
:1091B00000600000000006000000600000000006E3
:1091C00000000060000600000080020004000800AB
:1091D000100000020004000804000002000400085F
:1091E000001000200040008004000000FF7FFFFF0F
:1091F000FDFFFFFFFBFFFFFFF7FFFFFFEFFFFFFF9D
:10920000FFFDFFFFFFFBFFFFFFF7FFFFFBFFFFFF80
:10921000FFFDFFFFFFFBFFFFFFF7FFFFFFEFFFFF7C
:10922000FFDFFFFFFFBFFFFFFF7FFFFFFBFFFFFF32
:109230000102030405000203040500010304050004
:1092400001020500010203040405000102035505A3
:109250000010AA1A55250030AA3A0000AA0A55158E
:109260000020AA2A5535FF3F889200080000002000
:1092700024070000E806000878930008240700206F
:10928000B40900000C64000845020406082D010220
:1092900003040405440607080913A12B1B08B504A1
:1092A000211355152A40061908019713B53D1B08CF
:1092B000D9041AD5040131170206040501031480EC
:1092C00020FF8BAA0A02019C15AA0A55150008590D
:1092D00020AA2A5535FF3F0729030105040602038A
:1092E000127C1573FFFF04FF8080010125025B647F
:1092F00002130A13796712081201100C0504060202
:1093000003010103070505280B01020304020607F8
:109310000303040C3D0706040509191F191904313C
:109320000506064BAA1A024B381E026910312E4060
:10933000FD3969260211042F405F020C26405B268E
:109340002ACD55155515123902017F0316D0071A7B
:10935000FF01013B0261AA6C080108A80916C4912B
:10936000220312100A17401C12600A16901B0149B2
:08937000138D670200080000E4
:020000040800F2
:10FC00004A46545A594D46312D4E3330202020203B
:10FC1000050406020301AA0AAA0AAA0AAA0AAA0A4B
:10FC2000AA0ADE3F00100000FF0131000201664613
:10FC300000400040513800400040004000400101B9
:10FC400000400040FF387B257B257B25FF003333B8
:10FC50000201401F00016626B81E6626FFFFFFFF57
:10FC6000FFFF01010100010000000300000202008B
:04FC70000000AA5591
:04000005080000ED02
:00000001FF
